:100000000C9418050C9450050C9450050C94500554
:100010000C9450050C9450050C9450050C9450050C
:100020000C9450050C9450050C946A160C941F15F2
:100030000C94EC170C9450050C9450050C9450053E
:100040000C9450050C9450050C9471230C9450059D
:100050000C9450050C949F170C9450050C9450056B
:100060000C9450050C9450050C9450050C945005BC
:100070000C9450050C9450050C9450050C945005AC
:100080000C9450050C9450050C9450050C9450059C
:100090000C9450050C9450050C9450050C9450058C
:1000A0000C9450050C9450050C9450051106140640
:1000B000170621062406370641065606C006F20634
:1000C00004077E069106BC0ABC0AEE0AEE0A600B23
:1000D000080D080D080D7C0B5A0C6B0C6B0CB62729
:1000E000DD277529DD277529252848287529372911
:1000F0004A2900DA0281FFD9F1DB20A4A62EAF0045
:10010000A0C000A1C800AED580A81FD300408D14A8
:1001100020001E0F05643214783C1E1E140A0500D0
:100120002E808182838485868788898A8B8C8D8EB8
:100130008F9091929394A0A1A2A3A4A5A6A7A8A9E9
:10014000AAABACADAEAFB0B1B2B3B4C0C1C2C3C460
:10015000C5C6C7C8C9CACBCCCDCECFD0D1D2D3D4D7
:10016000006F666600206F6E0020436C69636B79D8
:100170003A006F666600206F6E00417564696F3AE1
:1001800000524742204C4947485420444953414279
:100190004C4544004853563A20002D2D2D2D2D2D31
:1001A0002D2D2D2D2D2D2D2D002020204C3A0053AE
:1001B000706C69744B422773205A696D6100222369
:1001C000252628292A2C2D2F3032333536383A3B34
:1001D0003D3E4042434547494A4C4E505153555786
:1001E000595A5C5E6062646668696B6D6F717375A5
:1001F00077797B7D7F81838587898A8C8E909294A5
:1002000096989A9C9E9FA1A3A5A7A8AAACAEAFB1B1
:10021000B3B4B6B8B9BBBCBEBFC1C2C3C5C6C7C9FB
:10022000CACBCCCDCED0D1D2D2D3D4D5D6D7D7D8B5
:10023000D9D9DADADBDBDBDCDCDCDCDCDDDDDDDD07
:10024000DCDCDCDCDCDBDBDBDADAD9D9D8D7D7D60F
:10025000D5D4D3D2D2D1D0CECDCCCBCAC9C7C6C5C6
:10026000C3C2C1BFBEBCBBB9B8B6B4B3B1AFAEAC0C
:10027000AAA8A7A5A3A19F9E9C9A98969492908EB7
:100280008C8A89878583817F7D7B79777573716F90
:100290006D6B6968666462605E5C5A59575553516C
:1002A000504E4C4A4947454342403E3D3B3A383622
:1002B000353332302F2D2C2A29282625232200AF32
:1002C00000AEA800015302535F00600061005C00B3
:1002D0005D005E0059005A005B00005C01000000F8
:1002E0001D5C1E5C0000205C0000235C255C00009F
:1002F000245CC35CC45C0100C65CC85CCA5CC75CAF
:10030000C95CCB5CE95CEB5CEF5C000101010101C5
:1003100001010101020202020202020202030303BE
:10032000030303030304040404040404050505058E
:10033000050606060606070707070708080808094E
:100340000909090A0A0A0B0B0B0C0C0C0D0D0D0EFA
:100350000E0E0F0F0F10101111111212131314148F
:10036000151516161717181819191A1A1B1B1C1D04
:100370001D1E1E1F2020212222232424252626275D
:100380002829292A2B2C2D2D2E2F3031323233348F
:1003900035363738393A3B3C3D3E3F404142434495
:1003A00045464748494A4C4D4E4F50515354555677
:1003B00058595A5B5D5E5F616264656668696B6C23
:1003C0006D6F7072737577787A7B7D7E808283859E
:1003D00087888A8C8E8F91939596989A9C9EA0A2DE
:1003E000A3A5A7A9ABADAFB1B3B5B7BABCBEC0C2E8
:1003F000C4C6C9CBCDCFD1D4D6D8DBDDDFE2E4E7AC
:10040000E9EBEEF0F3F5F8FAFDFFFFAA7F554005A2
:10041000010980A101850319012AB700150126B73A
:1004200000950175108100C0050C0901A10185042A
:1004300019012AA002150126A0029501751081005C
:10044000C005010906A101050719E029E7150025E6
:10045000019508750181029501750881010507194B
:100460000029FF150026FF00950675088100050884
:1004700019012905950575019102950175039101F1
:10048000C009023B00020100A0FA090400000103B8
:10049000010100092111010001224000070581032B
:1004A00008000109040100010300000009211101F5
:1004B0000001223200070582032000011201000220
:1004C000000000081D8D5BF70100010200010A0316
:1004D0005A0069006D006100000010037300700095
:1004E0006C00690074006B006200000004030904E2
:1004F00007087F0807003E5B4F5B3E003E6B4F6B7B
:100500003E001C3E7C3E1C00183C7E3C18001C57E4
:100510007D571C001C5E7F5E1C0000183C1800000C
:10052000FFE7C3E7FF00001824180000FFE7DBE740
:10053000FF0030483A060E00262979292600407F20
:1005400005050700407F05253F005A3CE73C5A005F
:100550007F3E1C1C0800081C1C3E7F0014227F22CA
:1005600014005F5F005F5F0006097F017F00006687
:1005700089956A0060606060600094A2FFA29400A8
:1005800008047E04080010207E20100008082A1CA1
:100590000800081C2A0808001E10101010000C1E6D
:1005A0000C1E0C0030383E383000060E3E0E0600A1
:1005B00000000000000000005F00000000070007CE
:1005C0000000147F147F1400242A7F2A12002313B2
:1005D00008646200364956205000000807030000F6
:1005E000001C224100000041221C00002A1C7F1C2C
:1005F0002A0008083E080800008070300000080843
:1006000008080800000060600000201008040200D4
:100610003E5149453E0000427F4000007249494931
:1006200046002141494D33001814127F1000274520
:10063000454539003C4A494931004121110907002B
:10064000364949493600464949291E000000140030
:10065000000000403400000000081422410014147F
:100660001414140000412214080002015909060064
:100670003E415D594E007C1211127C007F49494970
:1006800036003E41414122007F4141413E007F49C9
:10069000494941007F09090901003E414151730068
:1006A0007F0808087F0000417F4100002040413F53
:1006B00001007F08142241007F40404040007F023B
:1006C0001C027F007F0408107F003E4141413E0034
:1006D0007F09090906003E4151215E007F09192961
:1006E000460026494949320003017F0103003F408B
:1006F00040403F001F2040201F003F4038403F0047
:100700006314081463000304780403006159494D1D
:100710004300007F414141000204081020000041D5
:1007200041417F000402010204004040404040007B
:100730000003070800002054547840007F284444F8
:100740003800384444442800384444287F00385452
:100750005454180000087E09020018A4A49C7800D4
:100760007F080404780000447D4000002040403DA4
:1007700000007F102844000000417F4000007C04FE
:10078000780478007C080404780038444444380035
:10079000FC182424180018242418FC007C080404E5
:1007A000080048545454240004043F4424003C40AE
:1007B00040207C001C2040201C003C4030403C007D
:1007C0004428102844004C9090907C004464544C81
:1007D000440000083641000000007700000000419E
:1007E000360800000201020402003C2623263C00D9
:1007F000000000000000404040F0F8F8FF38FFF82B
:10080000F83FF8F8FF38FFF8F8F0404040000000EB
:1008100000000080C0C0C0800000C0C08000000098
:1008200080C0C000C0C0000080C0C0000000000048
:10083000C0C0C0C0C000C0C0000000000000000078
:1008400000000000000000000000000000000000A8
:100850000000000000000000000000000000000098
:10086000000000000000000000000000000000C0C8
:10087000F0F8FC3E1E06010000007F4141417F0070
:100880007F4141417F000080C0E07E5B4F5BFEC046
:100890000000C000DCD7DEDEDED7DC00C0000000D8
:1008A0000000000000000000000000000000000048
:1008B000000000000000494949FFFFFFFFE0DFBFE3
:1008C000BF00BFBFDFE0FFFFFFFF49494900000055
:1008D00000001F3F6060E0BF1F007F7F071E381EC3
:1008E000077F7F007F7F0E1F3B71600000000000CC
:1008F0007F7F0C0C0C007E7E007F7E0303007F7EDA
:1009000003037E7E03037F7E000F3E703C063C7037
:100910003E0F00327B49493F7E007F7E0303001E6D
:100920003F69696F2600000000000000000000031E
:100930000F1F3F3C7870600000007F4141417F0005
:100940007F4141417F00307B7F7830202030787FAD
:100950003B0003000F7F0F0F0F7F0F00030000000D
:100960000000000000000000000000000000000087
:10097000000000000000010101070F0F7F0F7F0F33
:100980000F7E0F0F7F0F7F0F0F0701010100000087
:100990000000000000000001010000000000000055
:1009A0000000000000000000000000000000000047
:1009B0000000000000000000000000000000000037
:1009C0000000000000000000000000000000000027
:1009D0000000000000000000000000000000000017
:1009E0000000000000000000000000000000000007
:1009F00000000000000000000000000000000000F7
:100A000000000000000000000000000000000000E6
:100A100000000000000000000000000000000000D6
:100A200000000000000000000000000000000000C6
:100A300011241FBECFEFDAE0DEBFCDBF04B603FE48
:100A400018C08091070690910806A0910906B09100
:100A50000A068730904BA740B04B59F41092070616
:100A6000109208061092090610920A06E0E0F8E3D8
:100A7000099512E0A0E0B1E0E6E5FBE602C00590D2
:100A80000D92A639B107D9F726E0A6E9B2E001C078
:100A90001D92A730B207E1F70E94FE0D0C94A93514
:100AA0000C9400008F929F92AF92BF92CF92DF92F0
:100AB000EF92FF920F931F93CF93DF93CDB7DEB7E3
:100AC0002A970FB6F894DEBF0FBECDBFFC01D080D1
:100AD000118183819481892B39F01F3F39F491E092
:100AE0000FEFD01203C003C091E001C090E090FF6F
:100AF00002C00C94EB0D7F0185E0DE01169601909B
:100B00000D928A95E1F7F70122818E819F81222340
:100B100049F00E944B2A082F682F8E819F810E94E6
:100B2000D32A03C00E94A72A082F812F90E0FC013E
:100B3000EE0FFF1FE80FF91F1CE0019FE00DF11DF4
:100B40001124ED0DF11DEE0FFF1FEE53FD4F05912A
:100B50001491F70182810032FCE51F0769F48823B4
:100B600009F451C36091AE0361FB992790F981E0CC
:100B7000892780FB61F90AC001322CE5120769F46C
:100B8000882309F440C36091AE0362606093AE03B2
:100B900087E090E00E94A32F36C302323CE51307A2
:100BA00061F48823E9F06091AE036D7F6093AE033A
:100BB00087E090E00E94A32F13C005322CE51207B6
:100BC00009F001C3882361F080E090E0ACEDB3E46C
:100BD0008093D4019093D501A093D601B093D7010F
:100BE0008091AE0380FF0DC081FF0BC0F7018281B1
:100BF000882339F0C8018E519C45029710F00E945D
:100C0000562DF7018281882309F411C1F801E75EAE
:100C1000FC45ED30F10508F00AC1EA5AFF4F0C948B
:100C200091320E941A1903C10E940B1900C18091D0
:100C3000170380FF03C00E940B1997C00E941A1966
:100C400094C00E94F218F3C080911703282F2695B4
:100C50002F5F2370922F990F897F892B8093170321
:100C6000233009F082C0897F809317037EC0809172
:100C7000180382FB222720F991E0922790FB82F94A
:100C80003AC020911703822F8695869586952091EC
:100C9000180323702295220F207E282B81E0820FDB
:100CA00030E02C373105A4F081E012C09091170399
:100CB000892F8695869586959091180393709295C5
:100CC000990F907E982B8FEF890F911101C08BE7C0
:100CD000282F220F220F220F909117039770922B2B
:100CE00090931703829586958770982F93708091C3
:100CF00018038C7F892B8093180337C04091180309
:100D0000242F26952695269530911903832F8370DD
:100D10008295880F807E982F922B892F90E00196E4
:100D200012C040911803242F2695269526953091C0
:100D30001903832F83708295880F807E982F922BC2
:100D4000892F90E00197282F220F220F220F477042
:100D5000422B4093180375E0969587957A95E1F7B5
:100D600083703C7F832B80931903609117037091EC
:100D700018038091190390911A030E94D51B57C044
:100D80008091190382FF10C08B7F809319036091BB
:100D90001703709118038091190390911A030E9410
:100DA000D51B60E081E01BC08460809319036091D3
:100DB0001703709118038091190390911A030E94F0
:100DC000D51B60E08CE00E94991964E182E00E94EA
:100DD000991965E081E00E94991961E08CE00E9418
:100DE000991925C090911903892F86958695869526
:100DF00090911A039295990F907E982B8AE0890F13
:100E0000983798F088E711C090911903892F86953B
:100E10008695869590911A039295990F907E982BBE
:100E200086EF890F943108F484E10E94A51980911E
:100E3000170380FF18C0F7012281982F96959370B1
:100E4000222379F0923078F4869586958695909154
:100E5000180393709295990F907E892B0E94CA195E
:100E600002C09111F1CF0E94D4176093B202709327
:100E7000B3028093B4029093B5020D31FCE51F07D5
:100E800039F4F7018281882371F10E94472DE3C272
:100E90000E31FCE51F0739F4F7018281882319F12F
:100EA0000E942D2DD8C20F31FCE51F0749F4F70130
:100EB00082818823C1F08091AE0380FDF1CFE5CF20
:100EC000C8018A529C45029708F0C9C1F701828186
:100ED000882349F01092B00364E070E084E091E070
:100EE0000E949D29B8C2F7018281882309F41CC29F
:100EF00010921D030430FDE51F0758F40B3F2CE54D
:100F0000120780F4C80182509C45449708F0F6C14E
:100F100009C002363DE5130729F0063A8DE51807AA
:100F200009F0ECC10E94DB1B90939E0280939D020E
:100F300001319CE5190709F4CEC008F045C009301D
:100F4000FCE51F0709F4A5C000F505303CE51307D3
:100F500009F48DC078F403309CE5190709F47FC0CB
:100F600008F081C002301C4509F01DC180919D022E
:100F7000816017C107302CE5120709F482C008F020
:100F800084C080919D0280610CC10D308CE51807F2
:100F900009F48DC070F40B30ECE51E0709F47FC036
:100FA00008F081C080919D028860846080939D02DA
:100FB000B3C00F302CE5120709F485C008F087C0D4
:100FC00080919D02877FEDC00E3F8CE5180709F4E4
:100FD00076C008F50531ECE51E0709F48EC068F40B
:100FE00003312CE5120709F47AC008F0B8C00E945A
:100FF000782B80919D028F77D4C00C3F8CE5180729
:10100000D1F108F058C00B3F1C4509F0CCC08091CD
:101010009E02816033C00230FDE51F0709F4ABC0BA
:1010200070F401153DE5130709F460C008F07EC0B7
:1010300080919E028260816080939E0284C002360D
:101040009DE5190709F49DC0063AEDE51E0709F470
:10105000A2C003301D4509F0A6C060E08DC080919C
:101060009D0282609EC080919D0284609AC08091A2
:101070009D02886096C080919E02826080939E024D
:1010800092C080919D0280628CC080919D0280649C
:1010900088C00E94782B80919D02806882C08091D8
:1010A0009D028E7F7EC080919D028D7F7AC080914F
:1010B0009D028B7F76C080919E028E7FDFCF8091D4
:1010C0009E028D7FDBCF80919D028F7E6AC08091D2
:1010D0009D028F7D66C080919D028F7B62C0809152
:1010E0009D02877F8B7F80939D021BC080919E0213
:1010F0008D7F8E7F80939E022BC080919D0282FB0C
:10110000222720F991E0922790FB82F990FB83F946
:1011100080939D02992329F064E070E084E691E0D9
:101120001BC062E070E084E391E016C080919E02F3
:10113000982F909591708E7F892B90FB81F98093E9
:101140009E02992329F064E070E084E491E004C0F9
:1011500062E070E084E291E00E949D2924C00E9438
:10116000782B80919D0287FB222720F991E092271E
:1011700090FB87F916C061E08EE090E00E94A32FFB
:1011800012C080919D0284FB222720F991E09227D2
:1011900090FB84F906C080919D02982F909590FB5A
:1011A00080F980939D0260919D0210919E0284E0DF
:1011B00090E00E94A32F612F82E290E00E94A32F73
:1011C0000E94782B48C103323CE51307E1F48823E1
:1011D00009F406CD29E038E348E95FE36091D401E2
:1011E0007091D5018091D6019091D7010E9404326F
:1011F0004B015C0120E030E84BEB54E40E94A73047
:1012000087FFEECC23C004328CE5180709F0E8CC48
:10121000F7018281882309F4E3CC29E038E348E927
:101220005FE36091D4017091D5018091D6019091D6
:10123000D7010E94AC304B015C0120E030E042E875
:1012400052E40E94FF3118160CF0CACC8092D401EF
:101250009092D501A092D601B092D701C1CC043FA3
:101260009CE5190749F406E221EE40EE64EF7CE5C7
:10127000C7010E946718EFC0053FECE51E07F8F4B0
:10128000093DFCE51F0731F407E225EE45EE69ED67
:101290007CE5EECF0A3D2CE5120731F408E221E0AF
:1012A00045EE6AED7CE5E4CF083D3CE5130709F027
:1012B0001ACE06E221EE41EE68ED7CE5D9CF063F7D
:1012C0008CE5180731F406E221EE42EE66EF7CE58C
:1012D000CFCF063F9CE5190730F407E225EE44EE38
:1012E00065EF7CE5C5CF073FECE51E0709F0FBCDB8
:1012F00007E225EE46EE67EF7CE5BACF0631FCE566
:101300001F0761F5809177038A7A91E009F490E0F4
:1013100090939802882311F065E301C069E28DE2A1
:1013200093E00E94151817C00631FCE51F0709F06D
:101330007BC080919802882309F4AAC385E3EDE27B
:10134000F3E023E333E09281891301C012823196E6
:101350002E173F07C1F70E946A1C7DC00B35FDE5C3
:101360001F0709F45BC058F401153CE51307C1F0F1
:101370000F3D1C4509F0A4C00E94F71B6CC00C3542
:101380009DE5190709F44CC00D351D4509F098C0BD
:1013900080919E0282FB882780F991E0892741C0D5
:1013A0000E94782B0E94E0178C0163E070E084E8D3
:1013B00091E00E949D29C8010E94C5178A3F9105AE
:1013C00038F48FE99FE00197F1F700C00000F3CFF8
:1013D0000E947A2281E08093E00080E28093D8002E
:1013E0001092C900EFE1FEE43197F1F700C0000070
:1013F00087E090EBDC018093070690930806A093AA
:101400000906B0930A069CE088E10FB6F894A89507
:10141000809360000FBE90936000FFCF81E001C019
:1014200080E00E94C31C4CC08091770382720C3C08
:101430002CE5120709F4B3C388F1013DECE51E0762
:1014400009F4C1C308F449C3053DECE51E0709F4DE
:10145000BDC308F055C380916D03877009F4BBC309
:10146000F7018281882309F4B6C380919E0282FD30
:10147000B2C382E02A960FB6F894DEBF0FBECDBF8E
:10148000DF91CF911F910F91FF90EF90DF90CF9060
:10149000BF90AF909F908F900C94A61C073C9CE54A
:1014A000190709F468C308F003C3043CFCE51F07EF
:1014B00009F457C308F0EEC2033C1C4509F42CC3E1
:1014C000F701828100811181882349F0C8010E94BF
:1014D0004B2AD82E682FC8010E94D32A04C0C80105
:1014E0000E94A72AD82E812F90E0FC01EE0FFF1F4B
:1014F000E80FF91F1CE0D19EE00DF11D1124E00F53
:10150000F11DEE0FFF1FEE53FD4F859194910E9448
:101510004C1A8C01982EF701D280A580A2946FE01E
:10152000A62280916D038770B9F0DD20A9F0812F8C
:10153000807F803421F080E2800F883068F08091D5
:101540009E0282FD09C082E00E94A61C80916D036C
:101550008770CC24C3948111C12CB12EB2943FE08A
:10156000B3228B2D90E08C30910508F051C2FC0124
:10157000ED59FF4F0C949132812F807F1F7088238B
:1015800011F01295107FDD20B9F0112309F42DC25E
:1015900080E2800F883010F0911006C080917703B0
:1015A000182B1093770305C080917603182B1093A6
:1015B00076030E946A1C19C2802F0E94832B11237C
:1015C00009F426C2005E083078F1992069F110957F
:1015D0008091760318231093760329C0812F807F92
:1015E0001F70803211F01295107F992021F0F1E0E8
:1015F0009F16D9F149C080919E0282FF1BC0DD2059
:1016000069F0112339F080917703182B1093770339
:101610000E946A1C80E00E94B42BFAC180E00E9404
:10162000832B112309F4F4C1812F0E94631C0E94B3
:101630006A1CEEC1DD2081F080917803AA2051F070
:1016400001E0A01207C0182B181709F4E1C110938C
:101650007803DEC1812B10C0AA2021F021E0A21660
:1016600009F4D6C10E945D1C27C0DD2041F035E0A1
:101670003A1508F4CDC1812F0E942E2AC9C184E0F9
:101680008A1508F4C5C118C0DD2049F0AA2099F3D5
:10169000F701858180FFA9C18F708583ECCFAA20D7
:1016A00059F0093309F0B1C1FFEF17EE23E0F15013
:1016B00010402040E1F7A7C1812F0E94442AA8C111
:1016C000812F86958695837019F0813059F0A0C1DD
:1016D000DD2019F0C801937002C080E090E00E9404
:1016E00045189CC1DD2019F0C801937002C080E04C
:1016F00090E00E942F1892C1812F837009F069C079
:10170000D1108AC1902F929596959770990F990F45
:10171000802F8F70882E912CA12CB12C092E04C003
:10172000880C991CAA1CBB1C0A94D2F704FF12C097
:101730004FE050E060E070E004C0440F551F661FAA
:10174000771F9A95D2F7DB01CA0180959095A095F5
:10175000B09503C080E090E0DC0116951695412F0E
:101760004370423019F1C8F40091790310917A0363
:1017700020917B0330917C03413059F088299929CD
:10178000AA29BB29BC01CD016023712382239323A5
:101790000AC0802A912AA22AB32ABC01CD01682955
:1017A00079298A299B290E944E2B36C1882999299B
:1017B000AA29BB290091790310917A0320917B0318
:1017C00030917C03BC01CD016027712782279327CC
:1017D000EACFDD2019F0812F817001C08695882322
:1017E00009F41AC1902F929596959770990F990FB9
:1017F000802F8F70882E912CA12CB12C092E04C023
:10180000880C991CAA1CBB1C0A94D2F704FF12C0B6
:101810004FE050E060E070E004C0440F551F661FC9
:10182000771F9A95D2F7DB01CA0180959095A09514
:10183000B09503C080E090E0DC0116951695412F2D
:1018400043704230D9F068F50091AE021091AF02BA
:101850002091B0023091B102413059F08829992984
:10186000AA29BB29BC01CD016023712382239323C4
:101870001EC0802A912AA22AB32A13C08829992936
:10188000AA29BB290091AE021091AF022091B002AB
:101890003091B102BC01CD016027712782279327C7
:1018A00006C0BC01CD01682979298A299B290E949B
:1018B000FE2AB2C01F70DD2039F0812F0E942D2B2F
:1018C000802F0E942E2AA8C0802F0E94442A812F98
:1018D0000E94082BA1C0802F32EF931609F443C059
:1018E000391538F090EF991659F0E1EF9E16B1F1E5
:1018F00077C0F3EF9F16F1F124EF921659F170C003
:10190000DD2019F134E03A1508F482C01F7181E03E
:1019100090E0A0E0B0E0AC01BD0104C0440F551F51
:10192000661F771F1A95D2F78091AE029091AF0291
:10193000A091B002B091B1028A019B01082719273A
:101940002A273B27C901B80129C025E02A1508F438
:101950005FC0DCCF80919E0282FF23C0DD2029F092
:10196000812F8F7130C0DD20D9F3812F8F710E94BC
:10197000082B4EC0DD2079F01F7181E090E0A0E0DF
:10198000B0E0BC01CD0104C0660F771F881F991F0E
:101990001A95D2F703C060E070E0CB010E94FE2AE6
:1019A00037C0DD2099F01F71812F0E942D2B80916F
:1019B0009E0282FD07C038E0139FC001112483609E
:1019C00080936D03812F0E942D2B22C081E00E9405
:1019D000A61C81E08A15E0F482E00E94A61C18C0D3
:1019E000DD2029F0AA2009F4BBCF802F14CEAA2035
:1019F00009F4BBCF893349F49FEFE7EEF3E0915050
:101A0000E040F040E1F700C00000802F0E94832BEF
:101A100088EF8B0D843010F40E945B18CC20A9F065
:101A200080916D0380FD11C0F70112828595859527
:101A300085950E942D2BC7010E94520580916D0350
:101A40008595859585950E94082B85E0F701DE0137
:101A5000119601900D928A95E1F789819A810E94F1
:101A6000A72A2A8130E0F901EE0FFF1F2E0F3F1F3A
:101A7000F9010CE0809FE00DF11D11248981E80F30
:101A8000F11DEE0FFF1FEE53FD4F85919491A3C002
:101A900089E255CC053C9CE5190709F467C0063C72
:101AA0001C4509F00DCD4FE052E268E172E280C0C2
:101AB000093CFCE51F0709F468C008F461C00A3C52
:101AC0003CE5130709F466C00B3C1C4509F0F8CC53
:101AD0004BEE51E26FED71E26BC00E3C2CE512074C
:101AE00009F469C008F460C00F3C8CE5180709F4DC
:101AF00067C0003D1C4509F0E3CC68E086E068C0A3
:101B0000063D2CE5120709F4A6CC0E351D4509F05B
:101B1000D7CC6EE189E15CC080910A0380FF1BC0D5
:101B20008E7F80930A0360910A0370910B0380916A
:101B30000C0390910D030E9451201092E1028FEF4F
:101B400090E7E2E081509040E040E1F700C0000003
:101B50000E94F71F80CC816080930A0361E0869524
:101B60002CC04CE552E265E672E222C045E652E244
:101B70006CE572E21DC048E152E26FE072E218C00B
:101B800047EF51E263E072E213C043E052E267EFD5
:101B900071E20EC04FED51E26BEE71E209C043E617
:101BA00050E264E770E204C044E750E263E670E2AA
:101BB0000E94EB1950CC61E081E00E9421224BCCC5
:101BC00065E082E005C06EE089E002C068E18FE078
:101BD0000E94D91940CC2A960FB6F894DEBF0FBEEA
:101BE000CDBFDF91CF911F910F91FF90EF90DF90CC
:101BF000CF90BF90AF909F908F900895CF93DF9339
:101C0000CDB7DEB76C970FB6F894DEBF0FBECDBF71
:101C100084B7877F84BF0FB6F894A8958091600041
:101C2000886180936000109260000FBE90E080E8B1
:101C30000FB6F89480936100909361000FBE85B752
:101C4000806885BF85B7806885BF87E09AE19093FB
:101C50009702809396020E9463150E940916809154
:101C6000E20084608093E200789480919503882359
:101C7000A1F01091E9001F709091EC00892F817004
:101C800090FD80E8182B1092E9008091E80083FD18
:101C90000E94D0261F701093E90082E084BD93E07B
:101CA00095BD9AEF97BD80936E0041E252E06DE2E0
:101CB00072E0A1E0B0E020E030E0FA01E20FF31FB3
:101CC00080818F3FA1F0E82FE295EF70F0E011A145
:101CD0008F707D0102C0EE0CFF1C8A95E2F7C701F0
:101CE0009E2D9095912391A392A1892B82A32F5F82
:101CF0003F4F2330310509F74D5F5F4F641775077C
:101D0000D1F684E0E2EAF2E0DF01E82E1D92EA94E7
:101D1000E9F7E9E9F2E0DF011D928A95E9F70E940F
:101D2000EC1B811102C00E94F71B82E090E00E9430
:101D30008F2F8093A6020E94DB1B90939E028093BC
:101D40009D0283E090E00E948F2F682F70E080E07A
:101D500090E00E944E2B0E94C12D0E94EC1B81112D
:101D600002C00E94F71B88E190E00E94972F6093C9
:101D70001703709318038093190390931A03672B2A
:101D8000682B692B11F40E94F2180E94072E67E05D
:101D900081E00E9499196CE886E10E94991963EE2E
:101DA00087E10E94991964E38AE10E94991969E127
:101DB0006F7D60688BE10E94991965EF8CE10E944C
:101DC000991960EA8DE10E94991960E38EE10E9401
:101DD000991961E083E00E94991961E08CE00E940A
:101DE000991960E081E00E94991960E08CE00E94FE
:101DF00099196FE084E00E94991961E08CE00E94DB
:101E0000991982E08093D70280E88093F2030E94C0
:101E1000072E6DE070E085E091E00E94A625892BF9
:101E200009F043C08091D70263E070E081FD3AC0C1
:101E300082E091E00E94A625892BB9F56DE070E063
:101E400082EF90E00E94A625892B79F50E94D41795
:101E5000DC01CB01805A9541AF4FBF4F80931103F6
:101E600090931203A0931303B0931403E5EFF3E0F0
:101E700080E092E0DF019C011D9221503040E1F7AB
:101E8000F093FC05E093FB058FEF9FEF9093F40335
:101E90008093F30381E080931603809315031092DF
:101EA000D80203C08FEF90E0C5CF80919F028111CF
:101EB00033C00E94EC1B811104C00E94F71B0E94DA
:101EC000852088E090E00E94972F60930A0370932A
:101ED0000B0380930C0390930D036E7F71F40E94AB
:101EE000852088E090E00E94972F60930A0370930A
:101EF0000B0380930C0390930D030E943E201092DD
:101F0000E10280910A0380FF04C060E086950E9490
:101F1000212281E080939F0224982C9A57985F9AFF
:101F20008FE891E00197F1F700C0000083B182953E
:101F3000817029B130E0220F232F221F330B232B76
:101F400011F490E001C092E0892B8093AD028CE9FE
:101F500091E09093210380932003CC24C39480913B
:101F60009503853009F07CC0B0E4FB2E00E112E15E
:101F700080919503853009F05CC080919503843091
:101F800009F445C0C092B6020E947A221092E10282
:101F90008091A102811116C0C092A10280910A0312
:101FA000982F91709093A0028E7F80930A039FEFE9
:101FB000A0E7B2E09150A040B040E1F700C00000BF
:101FC0000E94F71F0E94291910922403E8E1F0E013
:101FD0000FB6F894A895E09360000FBEF0926000F1
:101FE00083B7817F846083BF83B7816083BF789428
:101FF000889583B78E7F83BF0FB6F894A89580919C
:102000006000886180936000109260000FBE809134
:102010009403882309F4ACCF0E94171FE2EAF2E090
:1020200081918111A2C326EA32E02E173F07C1F742
:102030009FCF0E94782B0E945B181092A102809182
:10204000A002882349F080910A03816080930A03EB
:1020500060E086950E9421220E94F1191092B6023A
:102060000E94171FB82E81110E94D417E2EAF2E0F5
:10207000A7EAB2E000E010E0302F21919D91922775
:1020800021F180E0FF24F3944F2D4923D1F08F8775
:10209000388B2F2181E009F480E0898B0E94E017C2
:1020A0008160782F9B8B8A8B4F85588969898B89B2
:1020B0000E943B2CF801E955FD4F8081F826F08203
:1020C00019C08F5FFF0C8330F9F60F5F1F4F04308C
:1020D000110591F68FEF8C8B8D8B1E8A0E94E01775
:1020E0008160782F988F8F8B4C895D896E89888D60
:1020F0000E943B2C8091E102882309F470C09091EA
:10210000E002E0910A03E6958E2F891B8093DC02A2
:10211000923061F4E82FF0E0E55EFE4FE4910E2F7F
:1021200010E0ABE0EA2EA5E1FA2E34C0963061F45F
:10213000E82FF0E0E85EFE4FE4910E2F10E0FBEF99
:10214000EF2EF4E1FF2E26C0993069F4E82FE695D2
:10215000F0E0EB5EFE4FE4910E2F10E0E1EDEE2E8D
:10216000E4E1FE2E17C0993179F463E00E947132E8
:10217000E92FF0E0EE5EFE4FE4910E2F10E070E3E9
:10218000E72E74E1F72E06C000ED17E06CECE62EAA
:1021900063E1F62E8091DD02882361F01092DD026A
:1021A0000E94E0179093DB028093DA021092DF0224
:1021B0001092DE020E94E017E091DA02F091DB0259
:1021C0008E1B9F0B8F3F9F4750F40E0F1F1F1093C6
:1021D000DB020093DA028AED92E0F7010995809123
:1021E000AD02E82FEE0FEE0FE093AD0283B184FB5A
:1021F000222420F8312C99B1892F90E0880F892F63
:10220000881F990B009711F082E090E082299329B2
:102210008E2B8093AD028F70E82FF0E0E35DFD4FD1
:1022200090818091AC02890F8093AC02823064F07F
:102230008091AB028F5F8093AB0260E080E00E94F0
:10224000E32CDD24D39401C0D12C8091AC028F3FCC
:102250005CF48091AB0281508093AB0261E080E03E
:102260000E94E32CDD24D3948091AC02082E000C54
:10227000990B62E070E00E947D328093AC02D11035
:102280000E94D41780911603882309F45FC285EF5A
:1022900093E09093FC058093FB058091B602882320
:1022A00019F00E94291955C14091B2025091B30210
:1022B0006091B4027091B5022FB7F8948091250314
:1022C00090912603A0912703B09128032FBF841B70
:1022D000950BA60BB70B80339547A105B10508F008
:1022E000E1C00E944319809116038823A1F08091D8
:1022F000D802882381F062E070E08FE191E00E94D3
:10230000A625892B41F41092D8028FEF9FEF90936E
:10231000F4038093F3038FEA91E00E944F261A8E14
:10232000198E8091AE029091AF02A091B002B0914F
:10233000B102AD0166277727411551056105710589
:1023400021F0DB01CA0120E101C020E0492F5A2F12
:102350006B2F7727411551056105710519F0285F2D
:10236000DB01CA01AC01BD0104E076956795579584
:1023700047950A95D1F7411551056105710519F089
:102380002C5FDB01CA01AC01BD0112E076956795B7
:10239000579547951A95D1F7411551056105710576
:1023A00019F02E5FDB01CA01B695A7959795879521
:1023B000892B8A2B8B2B09F02F5F1F922F9380E1A3
:1023C00092E09F938F931F9282E08F938E01075E1E
:1023D0001F4F1F930F930E94B13289EA91E00E9430
:1023E0004F26C8010E945D268AE991E00E944F268F
:1023F00081E00E94691980910A030FB6F894DEBF4C
:102400000FBECDBF80FF26C084E991E00E944F2619
:1024100080910D031F928F9380910C031F928F93D5
:1024200080910B031F928F9383E192E09F938F9390
:102430001F928EE08F93085111091F930F930E94F2
:10244000B132C8010E945D260FB6F894DEBF0FBE00
:10245000CDBF07C081E891E00E944F2681E00E9435
:1024600069198AE791E00E944F268091AE0380FFB0
:1024700003C086E791E002C082E791E00E944F2608
:1024800089E691E00E944F268091AE0381FF05C04E
:1024900080FF03C085E691E002C081E691E00E94E2
:1024A0004F2657C04091B2025091B3026091B402DE
:1024B0007091B5022FB7F89480912503909126036F
:1024C000A0912703B09128032FBF841B950BA60B67
:1024D000B70B803C944DA140B10508F0E2CE0E94BC
:1024E000431981E291E00E944F2681E00E94691920
:1024F00080911603882369F18091F3039091F4038E
:10250000892B41F02091F3033091F403211531051B
:1025100029F501C18091D8028111F4CF198286E298
:102520008A831B821C821D8287E08E831F828FEF2D
:1025300088878FE2898724E630E049E050E0BE01D9
:102540006F5F7F4F88E70E94BE2E892B11F4C092E7
:10255000D802809116038111D5CFDDC08091D802B9
:102560008111D9C0482E512CEE24E394F12C082E71
:1025700002C0EE0CFF1C0A94E2F7A9014E215F2174
:10258000452B11F48F5FEECF9091D702920175E049
:10259000220F331F7A95E1F790FD12C08295880FC4
:1025A00080768093AA01220F232F221F330B3195AF
:1025B0002093AD01815E8093AB011092AE0112C0F9
:1025C00055E0369527955A95E1F7220F220F220FF5
:1025D0002093AA011092AD01295F2093AB0183E003
:1025E0008093AE0124E630E047E050E068EA71E015
:1025F00088E70E94BE2E892B09F08DC08091D702FA
:1026000080FD23C0C20145E0880F991F4A95E1F77C
:10261000AC014B505C4F04E610E020E230E060E497
:1026200088E70E94E52E892B09F075C00E944319A6
:10263000E094F0948091F3039091F403E822F9225E
:10264000F092F403E092F30366C080E2E7EBF2E07D
:10265000DF011D928A95E9F735E0440C551C3A9547
:10266000E1F7E1E4F2E0FC8FEB8F4DE352E0AB8D5C
:10267000BC8D8D91BC8FAB8FFA019191AF0182011E
:10268000090F111D0B501C4F90E089549D4FFC0108
:1026900027E0922E9F01281B390B7724739401C0E9
:1026A000770C2A95EAF7B801812CDB01AD90BD01CA
:1026B000A720292D28192770622E022E000C330B1B
:1026C000BA2D01C0BB0F6A94EAF76B2E31952195A4
:1026D00031092770332701C0A6942A95EAF76A28A2
:1026E000A0806A286082839428E08212DECF9A94C8
:1026F00031963FEF9312CECF85E492E0AB8DBC8D47
:102700008A179B0709F0B3CF04E610E020E230E01F
:1027100047EB52E084CF809115038823B9F00E94E3
:10272000D4170091110310911203209113033091DB
:102730001403DC01CB01801B910BA20BB30B8F3F69
:102740009F4FAF4FBF4710F40E942919B11001C02D
:10275000D1100E9443190E945B189091D9028917E9
:1027600009F4FDCB8093D902FACB09BD19BD09B498
:1027700000FEFDCF8091D8008F7D8093D80080919E
:10278000E00082608093E0008091E00081FDFCCF5A
:102790000E94782BEDCB08950895089580918A03C7
:1027A00008958093290370932B0360932A038091EB
:1027B0009503843001F582E08093E9008FEF9091DA
:1027C000E800815095FD06C095ED9A95F1F700005F
:1027D0008111F5CF8091E80085FF0DC040E050E009
:1027E00063E070E089E293E00E94A4268091E80013
:1027F0008E778093E8000895BC0184E00C94D11397
:10280000BC0183E00C94D113CF93DF9321E020939C
:10281000E9002FEF3091E800215035FD06C035ED7D
:102820003A95F1F700002111F5CF2091E80025FF3E
:1028300014C0EC0140E050E068E070E00E94A42683
:102840008091E8008E778093E80088E0FE01ABE895
:10285000B3E001900D928A95E1F7DF91CF91089551
:102860009F92AF92BF92CF92DF92EF92FF920F931F
:102870001F93CF93DF93FC01A280948081E0848337
:10288000EEEBF1E0B490EDE3F2E0E491C1EFD2E0E1
:10289000F2EEEF2EF2E0FF2ECC24CA94D12CEB19ED
:1028A0000E2F10E022E02A1530F080910B03888370
:1028B00080910C038983911003C01B821A8255C03A
:1028C0008B818823F9F081508B832FEF829FC00189
:1028D00011246C8170E00E94162FFB01FF27E25447
:1028E000FE4F8491E82FEB192FEFE29FC0011124D6
:1028F000B8010E94162F80910D03689FB00111242A
:102900007A8333C00E94762F20910D03269521589B
:1029100030E0A901440F551F322F2227240F351F05
:10292000232F33278217930704F582E08A1588F452
:102930000E94762FB6010E947D3288830E94762FF6
:1029400020910C032695622F70E00E947D32280FA3
:1029500029831A8280910D03843120F0893C18F07C
:1029600088EC01C084E18C838B8397014A81698163
:1029700088810E949420259623E0E20EF11C83E0DA
:10298000CA30D80709F08ECFDF91CF911F910F91F8
:10299000FF90EF90DF90CF90BF90AF909F900C94FE
:1029A000F71FEF92FF921F93CF93DF93EC0182EE1C
:1029B000E82E82E0F82E10E08C81970140910D0303
:1029C00060910C03810F0E9494201D5C83E0E80E4F
:1029D000F11C1F3F89F70E94F71F9A818C8190FF9D
:1029E00002C08F5F01C081508C83DF91CF911F9116
:1029F000FF90EF900895CF93DF93EC01EAE0F3E0CE
:102A0000438162818C810E942A218C818F5F8C831B
:102A1000DF91CF910895CF93DF93EC01EC81F0E04B
:102A2000E254FE4F4491EAE0F3E0628181810E942A
:102A30002A218C818F5F8C83DF91CF9108951F9223
:102A40000F920FB60F9211242F933F934F935F93E2
:102A50006F937F938F939F93AF93BF93CF93DF93A6
:102A6000EF93FF93C091E900CF708091EC00D82FD5
:102A7000D17080FDD0E81092E9008091F000877F4E
:102A80008093F00078940E94D0261092E900809103
:102A9000F00088608093F000CD2BCF70C093E900E8
:102AA000FF91EF91DF91CF91BF91AF919F918F9166
:102AB0007F916F915F914F913F912F910F900FBE3A
:102AC0000F901F901895E8EDF0E080818E7F808355
:102AD0001092E2001092DA001092E100A0EEB0E055
:102AE0008C9181608C9380818F77808319BCA7ED56
:102AF000B0E08C918E7F8C9380818F7E808310924A
:102B00002C0308952091E4003091E50095E6409172
:102B1000EC00842F817040FF23C08091E80080FD8D
:102B20001DC080919503882399F0853099F080919C
:102B3000EB0085FD11C04091E4005091E5002417A1
:102B4000350729F3915011F09A01E1CF84E00895FF
:102B500082E0089583E0089581E0089580E008957B
:102B60004091E80042FFDDCF08958091970387FFF1
:102B700011C08091E80082FD05C08091950381110C
:102B8000F8CF11C08091E8008B770BC0809195033E
:102B9000882349F08091E80080FFF8CF8091E80019
:102BA0008E778093E8000895982F973068F590937A
:102BB000E900981739F07091EC002091ED005091E8
:102BC000F00003C0242F762F50E021FD02C09F5F4C
:102BD000ECCF3091EB003E7F3093EB003091ED0075
:102BE0003D7F3093ED003091EB0031603093EB008E
:102BF0007093EC002093ED005093F0002091EE00D4
:102C000027FDE5CF80E008958F708093E90081E093
:102C10000895CF92DF92EF92FF920F931F93CF937D
:102C2000DF93C8EDD0E088818F7E8883E7EDF0E008
:102C300080818160808384E082BF81E080932C0367
:102C400088818E7F888302EE10E0F8011082109256
:102C5000DA0081EEC82ED12CF601108288818F77A0
:102C6000888388818068888388818F7D888319BC68
:102C7000109295031092960310929403109293036E
:102C800090EEE92EF12CF70180818B7F8083888183
:102C90008160888342E060E080E00E94D415F60104
:102CA00080818E7F8083F801808181608083808134
:102CB00088608083F70180818E7F80838881806136
:102CC0008883DF91CF911F910F91FF90EF90DF905C
:102CD000CF9008951F920F920FB60F9211242F9349
:102CE0003F934F935F936F937F938F939F93AF9394
:102CF000BF93EF93FF938091E10082FF09C0809121
:102D0000E20082FF05C08091E1008B7F8093E100AB
:102D10008091DA0080FF2AC08091D80080FF26C011
:102D20008091DA008E7F8093DA008091D90080FF55
:102D300018C080E189BD82E189BD09B400FEFDCFE4
:102D400081E08093950380912C0381110FC00E9434
:102D500063150E9409168091E20084608093E2006E
:102D600005C019BC1092950310922C038091E100CC
:102D700080FF17C08091E20080FF13C08091E200C5
:102D80008E7F8093E2008091E20080618093E20078
:102D90008091D80080628093D80019BC85E0809330
:102DA00095038091E10084FF30C08091E20084FFB0
:102DB0002CC080E189BD82E189BD09B400FEFDCF50
:102DC0008091D8008F7D8093D8008091E1008F7E24
:102DD0008093E1008091E2008F7E8093E2008091F9
:102DE000E20081608093E20080919603882311F0D5
:102DF00084E007C08091E30087FD02C081E001C04C
:102E000083E080939503809195038091E10083FF97
:102E100027C08091E20083FF23C08091E100877F7B
:102E20008093E10082E08093950310929603809155
:102E3000E1008E7F8093E1008091E2008E7F80939D
:102E4000E2008091E20080618093E20042E060E075
:102E500080E00E94D4158091F00088608093F0009B
:102E6000FF91EF91BF91AF919F918F917F916F9162
:102E70005F914F913F912F910F900FBE0F901F9038
:102E8000189520919D0330919E032617370748F02F
:102E90006115710539F42091E8002E772093E80040
:102EA00001C0B901FC0120E06115710579F1809143
:102EB00095038823F1F18530F1F18091E80083FDDD
:102EC0003CC08091E80082FD2EC08091E80080FF28
:102ED000EBCF2091F3008091F20090E0922B6115EE
:102EE000710551F08830910538F421912093F1005B
:102EF000615071090196F3CF21E0089709F020E0B5
:102F00008091E8008E778093E800CECF2111CFCF5B
:102F10000AC080919503882361F0853061F080912B
:102F2000E80083FD0AC08091E80082FFF2CF80E0D4
:102F3000089582E0089583E0089581E008957894EB
:102F40001F920F920FB60F9211248F939F93AF93FE
:102F5000BF938091250390912603A0912703B09100
:102F600028030196A11DB11D80932503909326038C
:102F7000A0932703B0932803BF91AF919F918F91A6
:102F80000F900FBE0F901F9018959C014FB7F894AB
:102F90008091250390912603A0912703B0912803E7
:102FA0004FBF821B930B08952FB7F89460912503B0
:102FB0007091260380912703909128032FBF0895D5
:102FC0002FB7F8948091250390912603A0912703B1
:102FD000B09128032FBF08951F920F920FB60F9242
:102FE00011248F939F93AF93BF93809124038111FA
:102FF00013C08091250390912603A0912703B091DF
:1030000028034196A11DB11D8093250390932603AB
:10301000A0932703B0932803BF91AF919F918F9105
:103020000F900FBE0F901F9018959C01FC013296D7
:103030009FEF80E04191461789F09F3F19F44111BD
:1030400001C0982F8F5F8630A9F79F3F39F0F901B3
:10305000E90FF11D97FDFA95628308950895209177
:103060002203309123032817390771F0909323032B
:1030700080932203E0912003F0912103309721F007
:103080000084F185E02D0994089520911E0330916C
:103090001F032817390771F090931F0380931E03B5
:1030A000E0912003F0912103309721F00680F78111
:1030B000E02D09940895E0912003F09121033097C9
:1030C00021F00190F081E02D099480E00895EF92C5
:1030D000FF920F93CF93DF93C42FD22FFC018281F5
:1030E0008823D1F040931D030E94E01790931C03A6
:1030F00080931B0380E28C0F883008F06DC0C7708E
:1031000081E001C0880FCA95EAF7DF91CF910F9156
:10311000FF90EF900C942E2A80911D0348134BC012
:1031200080911B0390911C030E94C517883C910558
:1031300008F041C0CD17C9F080E28C0F883040F410
:10314000C77081E001C0880FCA95EAF70E94442A3F
:1031500080E28D0F883048F481E09D2F977001C088
:10316000880F9A95EAF70E942E2A093319F0E12C6C
:10317000F12C03C080E5E82EF12C802F0E94B42BA7
:10318000E114F10451F08FE99FE00197F1F700C0DD
:10319000000091E0E91AF108F3CF802F0E94832B01
:1031A00080E28D0F8830C0F4D77081E001C0880FB5
:1031B000DA95EAF70AC080E28C0F883068F4C770AD
:1031C00081E001C0880FCA95EAF7DF91CF910F9196
:1031D000FF90EF900C94442ADF91CF910F91FF90D4
:1031E000EF90089589E780931703E8E1F3E0808189
:1031F0008470A9E1B3E09C919C7F9C9381608B7F5C
:103200008083609117037091180380911903909146
:103210001A030C94D51BE7E1F3E080818E7F808355
:1032200060911703709118038091190390911A030C
:103230000C94D51BE7E1F3E080818160808360918D
:103240001703709118038091190390911A030C943D
:10325000D51B8091160390911503882389F099233B
:1032600069F062E070E080EC92E00E94A625892B74
:1032700019F080911503089510921503909115038C
:1032800081E089270895809116038823F9F00E9430
:10329000D417DC01CB01805A9541AF4FBF4F8093CB
:1032A000110390931203A0931303B093140380911E
:1032B000150381110BC062E070E08EEB92E00E947A
:1032C000A625892B19F481E08093150380911503BD
:1032D0000895CF93E82F2091FB053091FC05255FE1
:1032E00033404091F203642F70E0C9010E94162F11
:1032F000481B842FEE2351F066E00E947132C82FE4
:10330000C150A8F080E20E94CF25FACFA901480F52
:10331000511D4115524018F080E020E030E0280FA8
:10332000311D2B503C4F3093FC052093FB05CF9172
:103330000895EFE0F3E08083618324E630E042E02B
:1033400050E0BF0184EB0C94BE2ECF93C82FE9E16F
:10335000F3E0982F990F990F990F80818770892B2F
:103360008083EAE1F3E09C2F929596959770808197
:10337000887F892B80836091170370911803809157
:10338000190390911A030E94D51B6C2F82E0CF91F4
:103390000C949919CF93C82F60E08CE00E94991982
:1033A0006C2F84E00E94991961E08CE0CF910C941D
:1033B000991990910A0390FF04C09695981740F0D0
:1033C00003C0811105C090E0961710F40C9465229B
:1033D00061E00C942122882311F0FA0101C0FB0165
:1033E000099460910A03669570E04BE050E08FEA23
:1033F00091E00E949732892B19F481E08093E102D9
:103400000E94E0179093DB028093DA02089580E037
:10341000089590919D0292FF0DC0282F28712830A9
:1034200019F4877F846006C0282F2471243011F49A
:103430008B7F886093FF0DC0282F2871283119F4E5
:10344000877E846106C0282F2471243111F48B7E7D
:10345000886120919E0220FF0DC0382F38713830CE
:1034600019F4877F816006C0382F3171313011F433
:103470008E7F886021FF0DC0282F2871283119F414
:10348000877E816106C0282F2171213111F48E7E43
:10349000886194FD877E0895CF93DF9382389105EC
:1034A00069F1B0F48133910509F46FC048F48932B1
:1034B000910509F465C08A32910509F46BC08AC090
:1034C0008533910509F457C089339105B9F082C05D
:1034D000833E910571F138F4803E9105B1F0823E52
:1034E000910511F177C0863E9105B9F1873E9105AE
:1034F000C9F1843E910509F06DC024C020919D0260
:1035000020FD53C021FD51C065C080919D0280FD0A
:1035100046C080919E0280FF48C080919D0284FD3C
:103520003FC183EE90E03EC180919D0282FF3AC090
:10353000F4CF80919D0282FD35C080919E0280FD76
:1035400034C0EBCF80919E0281FF35C080919D02F7
:1035500084FD26C187EE90E025C180919D0283FF06
:1035600027C0F4CF80919D0283FD22C080919E02EE
:1035700081FD21C0EBCF80919D0285FD1FC021C040
:1035800080919D0285FD1DC019C080919D0286FD20
:103590001BC01DC080919D0286FD19C015C089E326
:1035A00090E000C182EE90E0FDC080EE90E0FAC0B5
:1035B00086EE90E0F7C084EE90E0F4C089E290E0FF
:1035C000F1C085E390E0EEC08AE290E0EBC081E3D9
:1035D00090E0E8C0811532E5930708F069C08115D5
:1035E00041E5940728F0982F8827816F906ADAC008
:1035F000883E910568F5803E910508F0D3C0883A71
:103600009105B8F4853A910548F0855AE82FF0E025
:10361000EB5BFD4F808190E09064C4C081309105E8
:1036200009F4BBC008F4BCC08430910508F4B8C0EC
:10363000B9C08F3B910508F0B3C0885AE82FF0E07D
:10364000EE0FFF1FE85BFD4F808191819464AAC05B
:10365000811520E59207F0F09C0174E036952795DE
:103660007A95E1F7922F9370482F437021E030E074
:1036700002C0220F331F4A95E2F73C68392B8F7046
:10368000982F9695969540E2949FC0011124822B25
:10369000932B88C0811530E4930718F09F70906ACF
:1036A00081C09C013A9521153F4108F47BC078C048
:1036B000EC01C11586E5D807E8F5C11525E5D20767
:1036C00048F08C2F0E94091A8F7190E0982F88275C
:1036D000906268C0C11534E5D30728F09C2F882775
:1036E000846F906A5FC0AE01437055272C2F2695DA
:1036F0002695C115D34578F481E090E002C0880F8B
:10370000991F4A95E2F740E2249F90011124822BF1
:10371000932B9C6847C081E090E002C0880F991FFE
:103720004A95E2F740E2249F90011124822B932BCB
:103730009A6838C0C1152AE5D207F8F4C11539E5F1
:10374000D30790F08C2F8F700E94091A94E0D695C1
:10375000C7959A95E1F7CF70D0E0DC2FCC27D069E0
:103760009E01282BC9011EC0C11548E5D407C0F031
:103770009C2F8827806F906A15C0CE0190568115C6
:10378000904270F48D2F8F710E94091A282F2F718B
:10379000CE0199279062922B05C081E090E002C093
:1037A00080E090E0DF91CF910895AB01BC0188E10A
:1037B00090E00C94B52FCF9384E090E00E948F2F7F
:1037C000C82F82E290E00E948F2F2C2F30E0A901B9
:1037D000582BCA01CF91089580E090E00E949D2F60
:1037E00021E0893E9E4F09F020E0822F089569EE86
:1037F0007EEF80E090E00E94C12F60E082E090E0E8
:103800000E94A32F60E083E090E00E94A32F10921B
:10381000790310927A0310927B0310927C0360E08C
:1038200084E090E00E94A32F60E082E290E00E949A
:10383000A32F60E085E090E00E94A32F60E086E087
:1038400090E00E94A32F6FEF87E090E00E94A32FEB
:1038500040E050E0BA0188E090E00E94B52F60E0BF
:103860008DE090E00E94A32F40E050E0BA0188E193
:1038700090E00E94B52F60E087E190E00E94A32FC6
:1038800040E050E0BA018CE190E00E94B52F60E08A
:1038900070E080E290E00E94C12F0E94F21840E0A8
:1038A00050E0BA018FE090E00E94B52F40E050E078
:1038B000BA0183E190E00C94B52F809178038111D7
:1038C00010927803089580959091770389238093CF
:1038D000770308959091770380917603982B9093C6
:1038E0002D0380917803882389F0892B80932D0301
:1038F000EFE2F3E097E080E0915029F0219122235C
:10390000D9F38F5FF9CF81110E945D1C48E050E030
:103910006EE673E08DE293E00E94A432892BA9F059
:1039200088E0EDE2F3E0AEE6B3E001900D928A9517
:10393000E1F7E0912003F0912103309731F002800C
:10394000F381E02D8DE293E00994089520916D03B9
:103950008095822380936D03982F977099F430E0BF
:10396000482F082E000C550B2417350759F090915D
:103970009E0292FD07C08595859585950E94082B2E
:1039800010926D030895CF93C0919E02C2FB9927B8
:1039900090F9981799F080FBC2F9C0939E0260914C
:1039A0009D0284E090E00E94A32F6C2F82E290E0C1
:1039B0000E94A32F82E0CF910C94A61CCF91089572
:1039C00080916C0390913B03891719F08F5F87708A
:1039D000FBCF08950F931F93CF93DF9380913A030A
:1039E00082958F7009F05DC080913703882309F4B8
:1039F00058C080916C0310913B0360913503709126
:103A00003603C0913803D091390391E06F3F09F03C
:103A100090E0292F06E0811709F443C0209721F098
:103A20007F3F21F030E003C031E001C0322F90E051
:103A300030FD34C0089FF001099FF00D1124DF0113
:103A4000A45CBC4F11963C911197371327C03C9151
:103A5000361324C012963C91129731111FC0139651
:103A60004D915C9114974C1B5D0B483C5105B0F493
:103A700080913A038F70806180933A03EF5BFC4F33
:103A800080818F708061808385E393E00E9452057E
:103A9000DF91CF911F910F910C94E01C01968770DC
:103AA000BACFDF91CF911F910F910895CF93DF93FC
:103AB000D82FC92F0E944B2A2C2F30E0F901EE0F8E
:103AC000FF1F2E0F3F1FF9019CE0899FE00DF11DA4
:103AD0001124ED0FF11DEE0FFF1FEE53FD4F8591E9
:103AE00094910E944C1ADF91CF9108959F92AF92CA
:103AF000BF92CF92DF92EF92FF920F931F93CF93DB
:103B0000DF93CDB7DEB761970FB6F894DEBF0FBE77
:103B1000CDBF8C0185E0F801DE011D9601900D926C
:103B20008A95E1F7F801E2809091350360913603C0
:103B300040913803509139034115510531F06F3FE1
:103B400031F481E09F3F19F403C081E001C080E0BF
:103B5000F82FF1709F2E80FD1AC1F801308121816C
:103B6000C380D48085E3A82E83E0B82EF09037037D
:103B7000F601E41BF50BFF2009F4C6C080913A035F
:103B8000E83CF10508F091C0482F407F09F050C093
:103B9000621311C093130FC0FE2CE1100CC08F7084
:103BA000806180933A03C5010E94520580913A03D7
:103BB000F801858329C1CD2831F02F3F31F481E010
:103BC0003F3F19F403C081E001C080E080FD03C0E5
:103BD00081E08E2502C080E090E0F82FF170FF2E8A
:103BE00080FF1CC080916C0340913B0356E084171A
:103BF00009F4E8C090E0589FF001599FF00D11249E
:103C0000E45CFC4F6181261306C06081631303C02E
:103C10006281E61203C001968770E9CFFE2CEE2088
:103C200009F4F2C080913A03816080933A0349C05D
:103C3000621306C0931304C0E11002C0F80186C0ED
:103C4000C8010E94582B882351F1EE2041F12091A8
:103C50003A03822F82958F7090E0029774F08091E2
:103C600035039091360398878F831986DB86CA8641
:103C70002C87CE0107960E94520586E0F801A5E345
:103C8000B3E001900D928A95E1F70E94EA1C0AC008
:103C90006217C9F0C8010E94582B81111EC0C801CB
:103CA0000E945205FF24F394AFC0482F407F81F754
:103CB00085E393E00E94520586E0F50111928A9512
:103CC000E9F7F12CA1C09313E5CFE110E3CFF801A0
:103CD0008583C8010E94520554C0EE2001F3209153
:103CE0003A03822F82958F7090E0029734F2809190
:103CF0003503909136039A8389831B82DD82CC82BF
:103D00002E83CE010196B7CFE83CF105D0F5FE2C0D
:103D1000EE2029F2621327C0931325C020913A03A5
:103D200020FD18C0822F82958F70482F50E04115DA
:103D3000510581F0F80125834F30510541F08F5F27
:103D4000982F9295907F822F8F70892B8583C80141
:103D50000E94520586E0F801A5E3B3E001900D92C0
:103D60008A95E1F751C0C8010E94582B811185CF77
:103D700080913A03816080933A03C8010E94520502
:103D800043C086E0F50111928A95E9F73DC0EE2027
:103D900009F485CFC8010E94582BF82E882309F416
:103DA0007ECF86E0F801A5E3B3E001900D928A95FD
:103DB000E1F780913503909136030E94561D0E94D1
:103DC000EA1C22C03D872E878D859E850E94561D48
:103DD000292F22952F70223028F49F7039F08111FD
:103DE00005C00BC0243028F49F7049F4805E8830F1
:103DF00020F0C8010E9452059F2CF92C05C0F80143
:103E00009581907F99F7F9CF8F2D61960FB6F89431
:103E1000DEBF0FBECDBFDF91CF911F910F91FF90FD
:103E2000EF90DF90CF90BF90AF909F900895CF928A
:103E3000DF92EF92FF920F931F93CF93DF9300D007
:103E400000D0CDB7DEB719821A821B821C82CE0148
:103E500001966C0141E252E08DE2E82E82E0F82EFC
:103E6000B6018A01B3E0A0E031E0F80121918F01B1
:103E70002F3FA1F0822F82958F7090E0FC0180A1EE
:103E800090E02F7002C0959587952A95E2F780FD06
:103E900002C0832F02C080E090E0A82B330FB15006
:103EA00021F7F601A1936F014D5F5F4FE416F50610
:103EB000C1F644E050E089E992E00E94A43211E0AA
:103EC000009709F410E0892BA9F089819A81AB81D0
:103ED000BC818093990290939A02A0939B02B09325
:103EE0009C0281E080937F030E94E01790937E0301
:103EF00080937D0380917F038823D1F080917D039F
:103F000090917E030E94C517059790F080919902C9
:103F10008093A20280919A028093A30280919B02D7
:103F20008093A40280919C028093A50210927F034B
:103F3000812F0F900F900F900F90DF91CF911F91D5
:103F40000F91FF90EF90DF90CF900895CF92DF9286
:103F5000EF92FF926B017C0120E030E0A9010E940A
:103F6000A730811106C0809180008F7C80938000F3
:103F700039C080918000806280938000C09281036C
:103F8000D0928203E0928303F092840320E030E039
:103F900040E051E4C701B6010E9404329B01AC012C
:103FA00060E074E284E79BE40E94AC306B017C012A
:103FB0000E941E31709387006093860020E030E0FD
:103FC00048E452E4C701B6010E94043220E030E028
:103FD00048EC52E40E94AC300E941E3170938B007A
:103FE00060938A00FF90EF90DF90CF9008958091CA
:103FF0000A0380FF0AC0259A85B18F7D95B1906232
:104000002FB7F894E2EEF2E00BC0E2EEF2E011829C
:1040100010821282339632E0E13FF307C1F7EBCF13
:1040200032E0E13FF30789F0319148E095B90000B3
:1040300000C037FF85B9330F000000C000C000C0CA
:1040400085B900C04A9591F7EBCF2FBF8FE594E07B
:104050000197F1F700C00000089590910A0390FFC6
:104060000CC0E2EEF2E0818360834283339692E0FB
:10407000E13FF907C1F70C94F71F089580910A03F7
:10408000282F269530E02115310519F481708260C2
:1040900005C02F31310524F081708C6380930A03B1
:1040A0000895CF92DF92EF92FF926B017C010E9404
:1040B0003E20B701A60188E090E0FF90EF90DF90EE
:1040C000CF900C94B52F80910E03882319F0815066
:1040D00080930E0360910A0370910B0380910C038F
:1040E00090910D030C94512080910E03833018F4AD
:1040F0008F5F80930E0360910A0370910B03809190
:104100000C0390910D030C945120EAE0F3E083E05E
:10411000808311828FEF8283838314826081718117
:10412000828193810C945120AF92BF92CF92DF9203
:10413000EF92FF920F931F93CF93DF93E82EF62E0B
:10414000E901E42FF0E0611106C0E65FFC4FE49165
:104150004E2F2E2F71C0062F10E0E65FFC4F4491CA
:10416000F42FC42ED12C26E0829FC00111242FEF02
:1041700030E0B9010E94162F5BEA5603C001579F39
:10418000900D11248E0D911D8E0D911D582F550FE0
:10419000580FD901A01BB10BAC9DC001AD9D900D76
:1041A000BC9D900D1124E92FF59ED0011124AB2F59
:1041B000BB277901EA1AFB0AEC9CD001ED9CB00DFB
:1041C000FC9CB00D11245901A51AB108A09E7001E4
:1041D000A19EF00CB09EF00C1124EF2CFF242E19A0
:1041E0003F092C9D80012D9D100D3C9D100D11242B
:1041F000212F6230710591F048F461157105E1F0ED
:1042000061307105B9F4242F4B2F16C0643071054D
:1042100069F040F06630710579F00CC0242F492F09
:10422000E12F0AC0492FEF2F2B2F06C0292FE42F93
:10423000412F02C0292FEB2F49832883EA83DF9186
:10424000CF911F910F91FF90EF90DF90CF90BF9093
:10425000AF900895CF93DF9300D01F92CDB7DEB714
:1042600090910A0390FF0AC09E012F5F3F4F0E946A
:1042700094204B8169818A810E942D200F900F909C
:104280000F90DF91CF9108955F926F927F928F92FE
:104290009F92AF92BF92CF92DF92EF92FF920F93D5
:1042A0001F93CF93DF9300D01F92CDB7DEB7182FA7
:1042B000762E042F622E90910A0390FF6DC0E92F95
:1042C000E695AE2FB0E0AA58BD4F8C918093E002E6
:1042D0009E7F923061F49E012F5F3F4F812F0E949D
:1042E00094204B8169818A810E942D2043C08230B5
:1042F00019F400910D033EC0863019F410910B03A0
:1043000039C08930D9F38F30A9F5EF508E2F8170E5
:10431000582EE695F0E0E65FFB4FA590B49082EE54
:10432000C82E82E0D82EE12CF12CBB2495E0892EFA
:10433000912CAE9CC001AF9C900DBE9C900D1124A1
:10434000B4010E94162F812F511002C0860F01C0A8
:10435000861B9601402F672D0E9494208FEFE81A4C
:10436000F80A83E0C80ED11C85E0E816F10409F7CD
:104370000E94F71F10930B0370920C0300930D0320
:10438000662051F060910A0370910B0380910C0339
:1043900090910D030E9451200F900F900F90DF918C
:1043A000CF911F910F91FF90EF90DF90CF90BF9032
:1043B000AF909F908F907F906F905F900895EAE00C
:1043C000F3E0438128E0421B08F440E021E06281F1
:1043D00081810C944421EAE0F3E0438128E0420F1C
:1043E00008F44FEF21E0628181810C944421EAE0DE
:1043F000F3E0628128E0621B08F460E021E0438181
:1044000081810C944421EAE0F3E0628128E0620FAC
:1044100008F46FEF21E0438181810C944421EAE0AC
:10442000F3E0818121E04381628188500C94442132
:10443000EAE0F3E0818121E043816281885F0C94AE
:10444000442190910A0390FF36C09170811102C0FF
:10445000926006C08F3110F09C6302C0880F982BC9
:1044600090930A03662351F060910A0370910B0345
:1044700080910C0390910D030E94512060910A03DA
:10448000669570E04BE050E08FEA91E00E94973231
:10449000892B19F01092E10202C00E94F11981E00B
:1044A0008093DD0220E040910D0360910C03809128
:1044B0000B030C944421089580910A038695815042
:1044C00009F48EE161E00C94212280910A03869523
:1044D0008F5F8F3108F081E061E00C942122EFE6DC
:1044E000F0E080818B7F8083E0E8F0E080818F7C4A
:1044F000808308958091BA01811122C01092F10346
:104500000E946F221092AB031092AC031092A00392
:1045100010929F03E1EBF3E080E090E0A0E8BFEBB6
:104520001182108282839383A483B58317821682BB
:10453000389623E0E13FF20799F781E08093BA01D2
:1045400008957F928F929F92AF92BF92CF92DF9207
:10455000EF92FF920F931F93CF93DF934B015C0178
:104560006A018091AE0380FFAEC08091AD038111DE
:1045700002C00E94C12D20E030E0A901C501B401B4
:104580000E94A73087FF04C0B7FAB094B7F8B09480
:104590007090F103072D10E0E801219743E0000F30
:1045A000111F4A95E1F7E12CF12CCF3FFFEFDF0718
:1045B000D9F128E0E21AF108F801EE0DFF1DEF54E1
:1045C000FC4F2281338144815581C501B4010E9491
:1045D000A730811127C08E0133E0000F111F3A95DB
:1045E000E1F70F541C4F8091F10390E00197C81739
:1045F000D9070CF068C0219688E0F8013896D801F8
:1046000001900D928A95E1F70E94E017F8019187D9
:10461000808782869386A486B586D786C686085FFD
:104620001F4FE1CF2197C1CF81E0870D893020F561
:104630008093F10381E0809380038093AC03C09169
:10464000F103D0E021970E94E017FE0123E0EE0F76
:10465000FF1F2A95E1F7EF54FC4F918380838282FC
:104660009382A482B582D782C6820E94E01780918D
:10467000BA01882341F113C088E08093F10381EBF4
:1046800093E028E0FC013896DC0101900D922A9518
:10469000E1F7089623E0893E920799F7CBCF809106
:1046A0006F00846080936F008091800080628093AF
:1046B00080008091AC03882321F00E9477260E941D
:1046C000A61F1092BA01DF91CF911F910F91FF9019
:1046D000EF90DF90CF90BF90AF909F908F907F90A2
:1046E00008951F920F920FB60F9211242F923F92AE
:1046F0004F925F926F927F928F929F92AF92BF92F2
:10470000CF92DF92EF92FF920F931F932F933F93DD
:104710004F935F936F937F938F939F93AF93BF93C9
:10472000CF93DF93EF93FF9380918503909186035E
:10473000A0918703B09188030196A11DB11D8093BC
:10474000850390938603A0938703B09388036091B9
:1047500085037091860380918703909188030E945E
:104760004D316B017C0120E030E040E85CE360917A
:1047700081037091820380918303909184030E944E
:1047800004329B01AC01C701B6010E94A73087FD2E
:10479000BAC110928503109286031092870310927B
:1047A00088038091AC03811105C0C091AB03CC2379
:1047B00009F498C10E94E017EC018091AB038111CC
:1047C00002C0312CE4C08091A1039091A2030E9409
:1047D000C51720919F033091A0038217930788F398
:1047E0008091A1039091A2030E94C51720919F037D
:1047F0003091A0037C01E21AF30AD093A203C09384
:10480000A1030091A3031091A403C8010196909302
:10481000A4038093A3030E94E017A090A603B09086
:10482000A7038091A3039091A4038A159B0560F0D0
:10483000C091A503CC2329F01092A4031092A303E6
:1048400003C00E947A224EC18091AA03C091A303A3
:10485000D091A403C090A803D090A903811131C0C6
:10486000F80163E0EE0FFF1F6A95E1F7EC0DFD1D07
:10487000DE0173E0AA0FBB1F7A95E1F7AC0DBD1DF9
:104880002D913D914D915C916081718182819381E7
:104890000E94A730811115C081E08093AA034FE0E8
:1048A00050E060E070E0CB010E94A1221093A403CD
:1048B0000093A3038FE090E09093A00380939F0365
:1048C00064C01092AA038E0143E0000F111F4A95A5
:1048D000E1F70C0D1D1DF8016481758186819781BA
:1048E0000E941E319B01A0E6BAEE0E942B3020E010
:1048F0003EE140E050E00E940930F1E0AF1AB1081B
:10490000412C5EE1552E612C712C2E153F0550F087
:10491000D093A403C093A303E216F306E0F0C1E032
:10492000D0E01CC0085F1F4FCA15DB0588F7E21AEC
:10493000F30A2196F80164817581868197810E942E
:104940001E319B01A0E6BAEE0E942B30A30192011A
:104950000E940930DACFE901CE19DF098091A30363
:104960009091A40333E0880F991F3A95E1F7F6017F
:10497000E80FF91F6081718182819381AE010E94ED
:10498000A122D093A003C0939F033324339480913A
:10499000AC03882309F49EC08091AF03882311F0F3
:1049A0003324339401EB13E0812C912C412C512CB6
:1049B00020E8622E2FEB722E222423948091F103A3
:1049C00090E0881699060CF085C0F80186819781E1
:1049D00001978E3F9F4F08F077C0F8018081918149
:1049E0000E94C517F801268137818217930708F4C2
:1049F0006BC0C280D380E480F58020E030E0A90164
:104A0000C701B6010E94A73087FF04C0F7FAF094EF
:104A1000F7F8F0948091AC03882309F455C0809195
:104A2000AD03811102C00E94C12D91EBA92E93E02C
:104A3000B92EC7E0D0E0A7019601F50162AD73ADD4
:104A400084AD95AD0E94A730811126C083E0CC0FC4
:104A5000DD1F8A95E1F7CF54DC4F198218824A8214
:104A60005B826C827D821F821E8289EE93E08C17AE
:104A70009D07D9F088E0FE013896DE0101900D9285
:104A80008A95E1F7198618864A865B866C867D864C
:104A90001F861E862896E9CF219798E0A91AB108AB
:104AA000CF3FEFEFDE0739F60FC0209280038091F1
:104AB000F10381508093F103811106C00E946F229F
:104AC0002092BA011092AC03FFEF8F1A9F0A085F81
:104AD0001F4F74CFC0918003CC2319F01092800334
:104AE00001C0C32D8091AC03811107C08091AB033D
:104AF000811103C00E946F2206C0CC2321F00E94C6
:104B000077260E94A61FFF91EF91DF91CF91BF9171
:104B1000AF919F918F917F916F915F914F913F9155
:104B20002F911F910F91FF90EF90DF90CF90BF904A
:104B3000AF909F908F907F906F905F904F903F903D
:104B40002F900F900FBE0F901F901895EF92FF922D
:104B50000F931F93CF93DF93EC017B0164E670E02A
:104B600088E70E940D2E8C01EC0EFD1ECE15DF0590
:104B700061F017FD0AC0FE01849164E670E00E94B6
:104B80008E2E8C012196892B89F30E94122FC80149
:104B9000DF91CF911F910F91FF90EF900895CF93E8
:104BA000DF938A3011F481E003C08D3029F480E076
:104BB000DF91CF910C946919682F8091FB0590913A
:104BC000FC0526E0FC01A5EFB5E001900D922A95C9
:104BD000E1F7603E30F026E0FC0111922A95E9F7FA
:104BE0000AC0F6E06F9FB001112460517B4F46E090
:104BF00050E00E94862FC091FB05D091FC0546E055
:104C000050E0BE0185EF95E00E94A432892B49F166
:104C10009E01255F3340A90185E0569547958A9509
:104C2000E1F781E090E0BC0102C0660F771F4A9572
:104C3000E2F74091F3035091F403462B572B2B5F7F
:104C40003F4F65E0369527956A95E1F702C0880FDA
:104C5000991F2A95E2F7842B952B9093F403809368
:104C6000F3039E012F5E33404091F203642F70E006
:104C7000C9010E94162F481B463010F4240F311D25
:104C8000211582E0380710F020E030E02B503C4F37
:104C90003093FC052093FB05DF91CF910895CF93CE
:104CA000DF93EC01FE018491882321F00E94CF253F
:104CB0002196F8CFDF91CF9108950F931F93CF9353
:104CC000DF93EC01FC0101900020E9F78F01015016
:104CD0001109C017D10720F489910E94CF25F9CF7F
:104CE00081E0DF91CF911F910F910C946919CF92C0
:104CF000DF92EF92FF92E091F103EE23D9F0E150C1
:104D000088E0E802F0011124EF54FC4FC280D38008
:104D1000E480F58020E030E0A901C701B6010E94DF
:104D2000A73018163CF48091B003811106C0109290
:104D3000AF0303C0C12CD12C7601C701B601FF908F
:104D4000EF90DF90CF900895EF92FF920F931F9313
:104D5000CF93DF937C018B010E948215811119C0D2
:104D6000E70101151105A1F08091E80085FD0AC059
:104D70008091E8008E778093E8000E948215882356
:104D800081F307C089918093F10001501109E9CFA7
:104D900080E0DF91CF911F910F91FF90EF900895E8
:104DA0001F93CF93DF93CDB7DEB7AA970FB6F894D2
:104DB000DEBF0FBECDBFE7E9F3E08FE993E02091BE
:104DC000F10021938E179F07D1F7809198038330CC
:104DD00009F461C030F4813071F0823009F49BC075
:104DE000B2C08A3009F487C08B3009F46CC08930B6
:104DF00009F0A9C020C080919703813A09F0A3C0AF
:104E00008091E800877F8093E80080919B039091D8
:104E10009C03892B21F468E08BE893E003C060E0F9
:104E200080E090E070E00E9441178091E8008B776D
:104E30008093E80088C080919703813209F083C095
:104E400080919B0390919C03029708F07CC0809115
:104E5000E800877F8093E8008091E80082FD05C02C
:104E6000809195038111F8CF6EC02091F30080915D
:104E7000F20090E0922B029731F48091F1008130A2
:104E800011F0863021F48091F10080938A038091A3
:104E9000E8008B7754C080919703813A09F053C0A2
:104EA00080919B0390919C03892B09F04CC08091C9
:104EB000E800877F8093E8008091E80080FFFCCFC6
:104EC0008091BB0137C0809197038132E1F58091D9
:104ED0009B0390919C03892BB1F58091E800877F1B
:104EE0008093E8000E94B515809199038093BB01DF
:104EF0000E94782B28C080919703813221F5809100
:104F0000E800877F8093E8000E94B51580919A039E
:104F10008093890318C080919703813AA1F480910E
:104F2000E800877F8093E8008091E80080FFFCCF55
:104F3000809189038093F1008091E8008E778093BF
:104F4000E8000E94B5158091E80083FFCEC18091F2
:104F5000970390919803492F50E04A30510508F08B
:104F6000C4C1FA01E159FF4F0C949132803821F00D
:104F7000823809F0BAC108C08091930390919403DC
:104F8000992389F082600FC080919B038F708730D6
:104F900008F0ABC18093E9008091EB0085FB882786
:104FA00080F91092E9009091E800977F9093E800D3
:104FB0008093F1001092F10065C1282F2D7F09F038
:104FC00094C1882319F0823061F08FC180919903D8
:104FD000813009F08AC1933009F080E08093940316
:104FE0002EC08091990381112AC080919B038F70FC
:104FF0002FEF280F263008F078C18093E900209128
:10500000EB0020FF1CC0933021F48091EB00806204
:1050100014C09091EB0090619093EB0021E030E0A0
:10502000A90102C0440F551F8A95E2F74093EA0098
:105030001092EA008091EB0088608093EB00109260
:10504000E9008091E800877F20C181114EC1109155
:1050500099031F778091E3008078812B8093E30090
:105060008091E800877F8093E8000E94B5158091C9
:10507000E80080FFFCCF8091E30080688093E3002C
:10508000111102C082E001C083E0809395032DC11D
:105090008058823008F029C18091990390919A0339
:1050A0008C3D53E0950779F583E08A838AE2898312
:1050B0004FB7F894DE01139620E03EE051E2E32F73
:1050C000F0E050935700E49120FF03C0E295EF70A9
:1050D0003F5FEF708E2F90E0EA3010F0C79601C06E
:1050E000C0968D939D932F5F243149F74FBF8091D8
:1050F000E800877F8093E8006AE270E0CE010196C5
:105100000E944117AEC040919B0350919C03292FF0
:10511000332723303105A9F068F42130310509F433
:10512000F3C02230310509F0E0C08BE390E0E1E804
:10513000F4E044C02132310521F12232310571F110
:10514000D4C0992781309105A1F058F0029709F059
:10515000CCC0EEECF4E0E4918E2F90E0EEECF4E0C5
:105160002AC0ECEEF4E0E4918E2F90E0ECEEF4E057
:1051700022C0EAEDF4E0E4918E2F90E0EAEDF4E055
:105180001AC04115510509F4C4C04130510509F058
:10519000ACC089E090E0ECEAF4E010C041155105A4
:1051A00009F4BCC04130510509F09FC082E390E092
:1051B000EFE0F4E003C0009709F497C02091E80005
:1051C000277F2093E80020919D0330919E03821752
:1051D000930708F49C0140E02115310589F1809185
:1051E0009503882309F43DC08530D9F18091E8000A
:1051F00083FD37C08091E80082FD2FC08091E800D8
:1052000080FFEACF4091F3008091F20090E0942B70
:105210002115310559F08830910540F444914093AF
:10522000F1003196215031090196F2CF41E0089703
:1052300009F040E08091E8008E778093E800CCCFC1
:105240004111CDCF0AC080919503882351F085305C
:1052500041F08091E80083FD04C08091E80082FF66
:10526000F2CF8091E8008B778093E8003EC08038D1
:10527000E1F58091E800877F8093E80080919603B4
:105280008093F1008091E8008E778093E8000E947F
:10529000B5152BC0811129C08091990390919A0373
:1052A0009927029714F58091E800877F8093E800A2
:1052B00010919903109396030E94B515111106C021
:1052C0008091E30087FD02C081E001C084E080930B
:1052D000950342E061EC81E00E94D41542E261EC6A
:1052E00082E00E94D415809195038091E80083FFAD
:1052F0001AC08091E800877F8093E8008091EB00DE
:1053000080628093EB000FC082E190E0ECEBF4E070
:1053100055CF89E090E0E3E9F4E050CF80E490E0FD
:10532000E1E4F4E04BCFAA960FB6F894DEBF0FBECF
:10533000CDBFDF91CF911F910895CF92DF92EF9271
:10534000FF92CF93DF932091AE0320FD08C0DF9141
:10535000CF91FF90EF90DF90CF900C947A227B0159
:10536000EC018091AD03811102C00E94C12D80919A
:10537000AC0381110E947A2281E08093AB031092EA
:10538000AA03D093A903C093A803F092A703E092C5
:10539000A6031092A5031092A4031092A3036C819C
:1053A0007D818E819F810E941E319B01A0E6BAEE15
:1053B0000E942B30C12C2EE1D22EE12CF12CA70122
:1053C00096010E940930688179818A819B81A901B7
:1053D0000E94A1220E94E0179093A2038093A10350
:1053E0008091A8039091A903E091A303F091A403F5
:1053F00033E0EE0FFF1F3A95E1F7E80FF91F6481E4
:105400007581868197810E941E319B01A0E6BAEECC
:105410000E942B30A70196010E9409303093A0030F
:1054200020939F03DF91CF91FF90EF90DF90CF907B
:105430000895882341F08095909176038923809385
:1054400076030C946A1C0895882339F090917603B2
:10545000892B809376030C946A1C0895882339F075
:1054600090917703892B809377030C946A1C08959D
:1054700080E090E00E94451880E090E00E942F18A4
:10548000109276030C946A1C882321F00E94631CFE
:105490000C946A1C08958F929F92AF92BF92DF92F4
:1054A000EF92FF920F931F93CF93DF938090AE0202
:1054B0009090AF02A090B002B090B10240917903F9
:1054C00050917A0360917B0370917C03842A952A22
:1054D000A62AB72ACFE1D0E0292F30E08901000FBA
:1054E000111F020F131F2CE0D22EE82EF12CD50134
:1054F000C4010C2E04C0B695A795979587950A947C
:10550000D2F780FD04C0219790F780E014C0DC9EA4
:10551000F001DD9EF00D1124E00FF11FEE0DFF1DD7
:10552000EE0FFF1FEE53FD4F859194910E944C1A90
:10553000019749F38C2FDF91CF911F910F91FF902D
:10554000EF90DF90BF90AF909F908F900895292F9C
:10555000220F920F890F682F669566956695982F92
:10556000977085E0689FB001112440E050E080E032
:10557000FB01E40FF51FE350FA4F208130E0092EC4
:1055800002C0369527950A94E2F721703327042E3E
:1055900001C0220F0A94EAF7822B4F5F5F4F45301C
:1055A000510531F70895292F220F920F890FE82F07
:1055B000E695E695E695877051E001C0550F8A950E
:1055C000EAF785E0E89FF0011124E350FA4F20E06C
:1055D00030E070E04081CB01022E02C096958795A5
:1055E0000A94E2F78170819584278523842781932B
:1055F0002F5F3F4F2530310569F708956093AE0264
:105600007093AF028093B0029093B1020C94382A49
:105610000F931F9341E050E060E070E004C0440F3E
:10562000551F661F771F8A95D2F740955095609554
:1056300070958091AE029091AF02A091B002B091AE
:10564000B1028A019B01082319232A233B23C901A4
:10565000B8011F910F910C94FE2A0F931F9341E004
:1056600050E060E070E004C0440F551F661F771FD4
:105670008A95D2F78091AE029091AF02A091B002CC
:10568000B091B1028A019B01082B192B2A2B3B2BCD
:10569000C901B8011F910F910C94FE2A6093790300
:1056A00070937A0380937B0390937C030C94382A45
:1056B000FC01808191810E94561D92959F709630C9
:1056C00079F010F4925001C09A50923068F4803F03
:1056D00069F018F4883E40F409C0843F29F406C0FC
:1056E000883E20F0813F11F080E0089581E0089528
:1056F0001092770386E0EFE2F3E0DF011D928A95D6
:10570000E9F70C94382A882371F19CEF980F913AAD
:1057100060F4EDE2F3E09281891301C012823196C8
:1057200093E0E333F907B9F70DC090E2980F983092
:1057300058F4982F977081E001C0880F9A95EAF786
:105740000E94631C0C946A1C9BE5980F933020F414
:1057500080E090E00C944518885A873120F480E06E
:1057600090E00C942F180895CF93882309F453C028
:105770009CEF980F913AF8F4C82FEFE2F3E085E33D
:1057800093E02191C21721F08E179F07D1F70DC02A
:10579000EDE2F3E08281C81301C01282319643E04A
:1057A000E333F407B9F70E946A1C6C2F8DE293E093
:1057B0000E94151813C090E2980F983090F48770EB
:1057C00021E030E0A90102C0440F551F8A95E2F79D
:1057D000CA0190917703892B80937703CF910C9422
:1057E0006A1CEBE5E80FE33040F4F0E0EB5BFD4FC3
:1057F000808190E0CF910C944518885A873158F4F5
:10580000E82FF0E0EE0FFF1FE85BFD4F80819181F4
:10581000CF910C942F18CF9108959C013A952115A2
:105820003F4130F5DC01AA27B270AC014427547027
:105830009C012227387094FF0FC090FF02C080E1C6
:1058400001C080E0AB2B09F08062452B09F0806439
:10585000232B79F080680DC0892F8170AB2B09F064
:105860008260452B09F08460232B19F0886001C009
:1058700080E0FB0109941F93CF93DF93CDB7DEB790
:1058800067970FB6F894DEBF0FBECDBF4B8B5C8B16
:105890006D8B7E8B8F8B61111092760386E09E015B
:1058A000235F3F4FD901E82F1D92EA95E9F795E074
:1058B000FE017396D90101900D929A95E1F79C89AA
:1058C0004E895F897B897D879E876F87598B488B3F
:1058D000F901DE01179601900D928A95E1F7CE014C
:1058E00007960E94761D81113EC086E0FE01379624
:1058F000DE01119601900D928A95E1F7FF81E8850E
:105900006A857B856115710531F0EF3F31F481E0E7
:10591000FF3F19F403C081E001C080E080FD23C097
:1059200020913B0330E0C90101968770992740918F
:105930006C0350E08417950779F1F983EA837D833E
:105940006C8396E0929FD001939FB00D1124A45CCC
:10595000BC4FFE01319601900D929A95E1F780932C
:105960003B030E94E01C16E080916C0390913B0386
:105970008917F9F0189FC0011124845C9C4F0E9484
:10598000761D8823B1F080916C0390E001968770BA
:10599000992780936C03E8CF0E94782B10923B03E9
:1059A00010926C03E5E3F3E086E0DF011D928A9537
:1059B000E9F767960FB6F894DEBF0FBECDBFDF9153
:1059C000CF911F910895CF93C62F0E94D417609353
:1059D000B2027093B3028093B4029093B5028091A7
:1059E000AE0380FF03C081FD0E94562D80911703F6
:1059F00080FF0DC0982F96959695969580911803E7
:105A000083708295880F807E892B0E94CA1964E278
:105A10007AE2CC2379F089EA90E00E940D2C89EAA1
:105A20000E94B42B89EA0E94832B69E17AE289EA19
:105A300090E00EC08AEA90E00E940D2C8AEA0E9453
:105A4000B42B8AEA0E94832B69E17AE28AEA90E029
:105A50000E940D2C81E0CF91089562E070E080E01B
:105A600092E00E949D292FEF81EE94E0215080402A
:105A70009040E1F700C000000E947A226091AE03DE
:105A80006E7F6093AE0387E090E00C94A32F60914B
:105A9000AE0361606093AE0387E090E00E94A32FA5
:105AA00062E070E080EF91E00C949D29CF92DF924C
:105AB000EF92FF92CF93DF936091D4017091D50163
:105AC0008091D6019091D7019B01AC010E943B309F
:105AD0006B017C010E94762FCCEBD1E0BC01990FC9
:105AE000880B990B0E944F3120E03EEF4FEF56E4B8
:105AF0000E94AC302DEC3CEC4CE45DE30E9404329F
:105B000020E030E040E85FE30E943B30A7019601CF
:105B10000E940432688779878A879B870E94762F44
:105B2000BC01990F880B990B0E944F3120E03EEF8A
:105B30004FEF56E40E94AC302DEC3CEC4CE45DE3BE
:105B40000E94043220E030E040E85FE30E943B30F6
:105B50002091D4013091D5014091D6015091D701C7
:105B60000E940432688B798B8A8B9B8B63E070E098
:105B7000CE01DF91CF91FF90EF90DF90CF900C940A
:105B80009D298091AD03811141C00E94EC1B8111C0
:105B900002C00E94F71B87E090E00E948F2F809345
:105BA000AE03E1EBF3E080E090E0A0E8BFEB118210
:105BB000108282839383A483B583178216823896DA
:105BC00023E0E13FF20799F78091AD0381110CC00A
:105BD0000E946F22269A82E0809380008AE180935F
:105BE000810081E08093AD030E947A228091AE0310
:105BF00080FF06C063E070E088ED91E00E949D297F
:105C00000E94E0179093A2038093A103089510923D
:105C1000B9008CE08093B80008959F92AF92BF9234
:105C2000CF92DF92EF92FF920F931F93CF93DF9368
:105C3000B82EEB010E94E0176C01C431D10558F079
:105C4000CF3F8FEFD80759F0CE0164E170E00E949A
:105C5000162F7B0107C0EE24E394F12C03C025E04E
:105C6000E22EF12C84E8A82E94EA992E1092BC0022
:105C70009092BC000E94E0178C018091BC0087FDCF
:105C800008C00E94E017801B910B8E159F05A8F39A
:105C90002AC08091B900887F883041F08091B90096
:105CA000887F803119F00FEF1FEF1FC0B092BB004B
:105CB000A092BC000E94E0178C018091BC0087FD7F
:105CC00008C00E94E017801B910B8E159F05A8F35A
:105CD0000AC08091B900887F883111F0803419F7AB
:105CE00000E010E00EC00EEF1FEFCF3F8FEFD807A0
:105CF00009F4BCCFC6010E94C5178C179D0708F494
:105D0000B5CFC801DF91CF911F910F91FF90EF9018
:105D1000DF90CF90BF90AF909F9008950F931F9307
:105D2000CF93DF93EB018093BB0084E88093BC00AA
:105D30000E94E0178C018091BC0087FD0EC0CF3F10
:105D40008FEFD807C1F30E94E017801B910B8C17CF
:105D50009D0788F38EEF9FEF0CC02091B900287F3C
:105D600081E090E0283211F480E090E091958195F7
:105D70009109DF91CF911F910F910895CF92DF92FA
:105D8000EF92FF920F931F93CF93DF936B018A01E2
:105D90007901B9010E940D2EE6010C0D1D1DC017E1
:105DA000D10761F424E92093BC00DF91CF911F91CA
:105DB0000F91FF90EF90DF90CF90089597FDF2CF75
:105DC000B70189910E948E2EEACFCF92DF92EF9297
:105DD000FF920F931F93CF93DF93C62F6A01790130
:105DE000B8010E940D2E97FD11C0B8018C2F0E94A2
:105DF0008E2EE601EC0CFD1CCE15DF0539F097FD6B
:105E000005C0B80189910E948E2EF6CF24E9209317
:105E1000BC00DF91CF911F910F91FF90EF90DF9029
:105E2000CF90089584E98093BC000895AA1BBB1B02
:105E300051E107C0AA1FBB1FA617B70710F0A61B8A
:105E4000B70B881F991F5A95A9F780959095BC01AB
:105E5000CD0108958F929F92AF92BF92CF92DF9221
:105E6000EF92FF92CF93DF93EC01688179818A8171
:105E70009B81611571058105910521F464E279ED3D
:105E80008BE597E02DE133EF41E050E00E94D72F02
:105E900049015A019B01AC01A7EAB1E40E94F62F27
:105EA0006B017C01ACEEB4EFA50194010E940430BB
:105EB000DC01CB018C0D9D1DAE1DBF1DB7FF03C0C6
:105EC0000197A109B04888839983AA83BB839F77F0
:105ED000DF91CF91FF90EF90DF90CF90BF90AF9088
:105EE0009F908F9008950E942A2F089580E091E05E
:105EF0000E942A2F0895A0E0B0E0809300019093C3
:105F00000101A0930201B09303010895FB01DC019C
:105F100002C005900D9241505040D8F70895F9996C
:105F2000FECF92BD81BDF89A992780B50895A6E16C
:105F3000B0E044E050E00C94C92FA8E1B0E042E0AA
:105F400050E00C94C92F262FF999FECF92BD81BD48
:105F5000F89A019700B4021639F01FBA20BD0FB6A7
:105F6000F894FA9AF99A0FBE08950396272F0E9483
:105F7000A42F0E94A32F252F0E94A42F242F0C941E
:105F8000A42F0196272F0E94A42F0C94A32FDC018D
:105F9000CB01FC01F999FECF06C0F2BDE1BDF89A34
:105FA000319600B40D9241505040B8F70895052E37
:105FB00097FB1EF400940E94EE2F57FD07D00E941D
:105FC000093007FC03D04EF40C94EE2F5095409509
:105FD000309521953F4F4F4F5F4F08959095809595
:105FE000709561957F4F8F4F9F4F08950E942B3082
:105FF000A59F900DB49F900DA49F800D911D11241D
:106000000895B7FF0C94F62F0E94F62F821B930B76
:106010000895A1E21A2EAA1BBB1BFD010DC0AA1FE9
:10602000BB1FEE1FFF1FA217B307E407F50720F001
:10603000A21BB30BE40BF50B661F771F881F991F7C
:106040001A9469F760957095809590959B01AC01C5
:10605000BD01CF010895A29FB001B39FC001A39FCE
:10606000700D811D1124911DB29F700D811D112491
:10607000911D08955058BB27AA270E9452300C94B6
:10608000C5310E94B73138F00E94BE3120F039F49A
:106090009F3F19F426F40C94B4310EF4E095E7FB1D
:1060A0000C94AE31E92F0E94D63158F3BA1762072B
:1060B00073078407950720F079F4A6F50C94F8315E
:1060C0000EF4E0950B2EBA2FA02D0B01B901900113
:1060D0000C01CA01A0011124FF27591B99F0593F57
:1060E00050F4503E68F11A16F040A22F232F342F9F
:1060F0004427585FF3CF469537952795A795F040ED
:106100005395C9F77EF41F16BA0B620B730B840B01
:10611000BAF09150A1F0FF0FBB1F661F771F881FB9
:10612000C2F70EC0BA0F621F731F841F48F4879511
:1061300077956795B795F7959E3F08F0B0CF939503
:10614000880F08F09927EE0F9795879508950E947C
:106150008A3108F481E008950E94C0300C94C53162
:106160000E94BE3158F00E94B73140F029F45F3FE1
:1061700029F00C94AE3151110C94F9310C94B431D6
:106180000E94D63168F39923B1F3552391F3951BFF
:10619000550BBB27AA2762177307840738F09F5F48
:1061A0005F4F220F331F441FAA1FA9F335D00E2EB5
:1061B0003AF0E0E832D091505040E695001CCAF722
:1061C0002BD0FE2F29D0660F771F881FBB1F2617E5
:1061D00037074807AB07B0E809F0BB0B802DBF01BC
:1061E000FF2793585F4F3AF09E3F510578F00C948B
:1061F000AE310C94F9315F3FE4F3983ED4F38695C9
:1062000077956795B795F7959F5FC9F7880F911DAB
:106210009695879597F90895E1E0660F771F881F97
:10622000BB1F621773078407BA0720F0621B730B4A
:10623000840BBA0BEE1F88F7E09508950E94DE31BB
:1062400088F09F5798F0B92F9927B751B0F0E1F037
:10625000660F771F881F991F1AF0BA95C9F714C0E7
:10626000B13091F00E94F831B1E008950C94F8310A
:10627000672F782F8827B85F39F0B93FCCF3869520
:1062800077956795B395D9F73EF49095809570957D
:1062900061957F4F8F4F9F4F0895E89409C097FBFA
:1062A0003EF490958095709561957F4F8F4F9F4FED
:1062B0009923A9F0F92F96E9BB279395F695879531
:1062C00077956795B795F111F8CFFAF4BB0F11F4F4
:1062D00060FF1BC06F5F7F4F8F4F9F4F16C088239B
:1062E00011F096E911C0772321F09EE8872F762FD1
:1062F00005C0662371F096E8862F70E060E02AF012
:106300009A95660F771F881FDAF7880F96958795FD
:1063100097F90895990F0008550FAA0BE0E8FEEFD2
:1063200016161706E807F907C0F012161306E40759
:10633000F50798F0621B730B840B950B39F40A2652
:1063400061F0232B242B252B21F408950A2609F430
:10635000A140A6958FEF811D811D089597F99F6734
:1063600080E870E060E008959FEF80EC08950024DD
:106370000A941616170618060906089500240A94AA
:1063800012161306140605060895092E0394000C30
:1063900011F4882352F0BB0F40F4BF2B11F460FFBF
:1063A00004C06F5F7F4F8F4F9F4F089557FD9058E8
:1063B000440F551F59F05F3F71F04795880F97FBC9
:1063C000991F61F09F3F79F0879508951216130683
:1063D0001406551FF2CF4695F1DF08C016161706B2
:1063E0001806991FF1CF86957105610508940895E7
:1063F000E894BB2766277727CB0197F908950E9479
:106400008A3108F48FEF08950E9417320C94C53139
:106410000E94B73138F00E94BE3120F0952311F070
:106420000C94AE310C94B43111240C94F9310E94C7
:10643000D63170F3959FC1F3950F50E0551F629FC1
:10644000F001729FBB27F00DB11D639FAA27F00DCD
:10645000B11DAA1F649F6627B00DA11D661F829FF4
:106460002227B00DA11D621F739FB00DA11D621FD9
:10647000839FA00D611D221F749F3327A00D611DF6
:10648000231F849F600D211D822F762F6A2F1124D8
:106490009F5750409AF0F1F088234AF0EE0FFF1F0B
:1064A000BB1F661F771F881F91505040A9F79E3F62
:1064B000510580F00C94AE310C94F9315F3FE4F358
:1064C000983ED4F3869577956795B795F795E795B8
:1064D0009F5FC1F7FE2B880F911D9695879597F9C1
:1064E0000895991B79E004C0991F961708F0961B30
:1064F000881F7A95C9F78095089597FB072E16F4A3
:10650000009407D077FD09D00E94162F07FC05D014
:106510003EF4909581959F4F0895709561957F4FBA
:106520000895EE0FFF1F0590F491E02D0994FC01F2
:106530004150504030F001900616D1F73197CF010D
:106540000895882799270895FB01DC0104C08D91E7
:106550000190801921F441505040C8F7881B990BD5
:106560000895AEE0B0E0E7EBF2E30C9480350D89DE
:106570001E898F89988D26E02C831A83098397FFC3
:1065800002C080E090E801979E838D83AE01455E56
:106590005F4F698D7A8DCE0101960E94E1324D8167
:1065A0005E8157FD0AC02F813885421753070CF4CE
:1065B0009A01F801E20FF31F10822E96E4E00C948A
:1065C0009C35ABE0B0E0E7EEF2E30C9472356C0181
:1065D0007B018A01FC0117821682838181FFCCC175
:1065E000CE0101963C01F6019381F70193FD85915F
:1065F00093FF81917F01882309F4BAC1853239F470
:1066000093FD859193FF81917F01853229F4B60135
:1066100090E00E94D834E7CF912C212C312CFFE15F
:10662000F315D8F08B3279F038F4803279F0833278
:10663000A1F4232D20611DC08D3261F0803369F4F7
:10664000232D216016C0832D8260382EE32DE46057
:106650003E2E2AC0F32DF8601DC037FC2DC020ED62
:10666000280F2A3040F08E32B9F436FC81C1232D38
:106670002064322E19C036FE06C08AE0989E200D96
:106680001124922E11C0EAE02E9E200D1124222EFC
:10669000F32DF0623F2E08C08C3621F4832D8068E4
:1066A000382E02C0883641F4F70193FD859193FF9F
:1066B00081917F018111B3CF982F9F7D95549330A5
:1066C00028F40C5F1F4F9FE399830DC0833631F090
:1066D000833771F0833509F059C021C0F8018081FA
:1066E00089830E5F1F4F88248394912C530113C01C
:1066F0002801F2E04F0E511CF801A080B18036FE57
:1067000003C0692D70E002C06FEF7FEFC5010E94EA
:10671000CD344C018201F32DFF773F2E16C02801A6
:1067200022E0420E511CF801A080B18036FE03C069
:10673000692D70E002C06FEF7FEFC5010E94C23487
:106740004C01F32DF0683F2E820133FC1BC0822DDB
:1067500090E088169906B0F4B60180E290E00E94BD
:10676000D8342A94F4CFF50137FC859137FE819116
:106770005F01B60190E00E94D83421102A9421E0F4
:10678000821A91088114910471F7E8C0843611F0DF
:10679000893641F5F80137FE07C060817181828139
:1067A00093810C5F1F4F08C060817181072E000C20
:1067B000880B990B0E5F1F4FF32DFF763F2E97FF2F
:1067C00009C090958095709561957F4F8F4F9F4F31
:1067D000F0683F2E2AE030E0A3010E941435882E95
:1067E000861845C0853731F4232D2F7EB22E2AE03E
:1067F00030E025C0932D997FB92E8F36C1F018F463
:10680000883579F0B5C0803719F0883721F0B0C0ED
:10681000E92FE061BE2EB4FE0DC0FB2DF460BF2E4B
:1068200009C034FE0AC0292F2660B22E06C028E017
:1068300030E005C020E130E002C020E132E0F801A4
:10684000B7FE07C060817181828193810C5F1F4F09
:1068500006C06081718180E090E00E5F1F4FA30150
:106860000E941435882E8618FB2DFF773F2E36FEAA
:106870000DC0232D2E7FA22E891458F434FE0BC098
:1068800032FC09C0832D8E7EA82E05C0B82CA32C07
:1068900003C0B82C01C0B92CA4FE0FC0FE01E80D46
:1068A000F11D8081803321F49A2D997EA92E09C093
:1068B000A2FE06C0B394B39404C08A2D867809F072
:1068C000B394A3FC11C0A0FE06C0B21488F4280C37
:1068D000922C9B180EC0B21460F4B60180E290E0D6
:1068E0000E94D834B394F7CFB21418F42B1802C016
:1068F000982C212CA4FE10C0B60180E390E00E94E9
:10690000D834A2FE17C0A1FC03C088E790E002C003
:1069100088E590E0B6010CC08A2D867859F0A1FE7A
:1069200002C08BE201C080E2A7FC8DE2B60190E0DC
:106930000E94D834891438F4B60180E390E00E94B4
:10694000D8349A94F7CF8A94F301E80DF11D808131
:10695000B60190E00E94D8348110F5CF222009F4CE
:1069600042CEB60180E290E00E94D8342A94F6CF5D
:10697000F6018681978102C08FEF9FEF2B96E2E1AF
:106980000C948E35FC010590615070400110D8F7D1
:10699000809590958E0F9F1F0895FC016150704067
:1069A00001900110D8F7809590958E0F9F1F089544
:1069B0000F931F93CF93DF93FB01238121FD03C02E
:1069C0008FEF9FEF2CC022FF16C046815781248194
:1069D00035814217530744F4A081B1819D012F5F97
:1069E0003F4F318320838C93268137812F5F3F4F28
:1069F0003783268314C08B01EC01FB010084F185F1
:106A0000E02D0995892BE1F6D80116968D919C9180
:106A10001797019617969C938E931697CE01DF9148
:106A2000CF911F910F910895FA01AA27283051F1B3
:106A3000203181F1E8946F936E7F6E5F7F4F8F4FAF
:106A40009F4FAF4FB1E03ED0B4E03CD0670F781F0E
:106A5000891F9A1FA11D680F791F8A1F911DA11DF3
:106A60006A0F711D811D911DA11D20D009F468942C
:106A70003F912AE0269F11243019305D3193DEF6D4
:106A8000CF010895462F4770405D4193B3E00FD08A
:106A9000C9F7F6CF462F4F70405D4A3318F0495D75
:106AA00031FD4052419302D0A9F7EACFB4E0A69558
:106AB0009795879577956795BA95C9F7009761057A
:106AC000710508959B01AC010A2E069457954795D0
:106AD00037952795BA95C9F7620F731F841F951FC5
:106AE000A01D08952F923F924F925F926F927F92D6
:106AF0008F929F92AF92BF92CF92DF92EF92FF92CE
:106B00000F931F93CF93DF93CDB7DEB7CA1BDB0B79
:106B10000FB6F894DEBF0FBECDBF09942A8839881E
:106B200048885F846E847D848C849B84AA84B98425
:106B3000C884DF80EE80FD800C811B81AA81B98131
:106B4000CE0FD11D0FB6F894DEBF0FBECDBFED0145
:066B50000895F894FFCF48
:106B56000100000000005C44000080415C978A440C
:106B66000000804152D0A444000080410000DC4473
:106B76000000804100005C440000004100005C44CD
:106B86000000004100005C440000004100005C443D
:106B96000000004148F176440000C04000005C441B
:106BA6000000C04048F176440000C04000005C444C
:106BB6000000C04048F176440000C04000005C443C
:106BC6000000C04048F176440000C04000005C442C
:106BD6000000C04052D02445000000410000DC44C3
:106BE6000000004152D0A44400004041CE130414DA
:106BF600CD130014FC13CB130021007F22000301E8
:106C06000F101112131415161718010100008242F5
:106C16000000803F0000DC43000040400000DC43F1
:106C26000000803F0000DC4352D0A4440000004135
:106C36000000DC440000004152D0244500004041E1
:106C460000005C44000000410000DC4400000041FC
:106C56000000DC440000004100005C4400000041EC
:106C66002564002533642C202533642C20253364C9
:106C76000066969567F794C6F5F6F0F1F400FF0105
:106C860000010000FFFF0000010001FF00000810E6
:106C96001818100800818283E200E900EA00B500B6
:106CA600B600B700CD008301CC008A0192019401A1
:106CB6002102230224022502260227022A02B30009
:106CC600B4006F0070000001020202020606060907
:106CD60009090909090F0F0F0F0F0F0F0F0F0F19D2
:066CE6001919191919002B
:00000001FF
